:020000040800F2
:1030000018190020C931000893980008614F000882
:1030100091980008713800080BAC0008000000000F
:1030200000000000000000000000000031A30008C4
:10303000034200080000000049A000082DA6000877
:10304000E3310008E3310008E3310008E331000810
:10305000E3310008E3310008E3310008E331000800
:10306000E3310008E3310008E3310008854000083F
:10307000E3310008E3310008E3310008E3310008E0
:10308000E3310008E331000801350008E3310008AE
:103090005DAB0008E3310008E3310008E3310008CC
:1030A00079A60008C9A60008E3310008E33100084A
:1030B00011A70008E331000859A70008E331000810
:1030C000E3310008E3310008E3310008E331000890
:1030D000E3310008F9AA0008FDAA0008E33100085E
:1030E000E3310008E3310008E331000800F002F8A2
:1030F00000F05AF80AA090E8000C82448344AAF138
:103100000107DA4501D100F04FF8AFF2090EBAE835
:103110000F0013F0010F18BFFB1A43F0010318470B
:10312000E89A0000089B00000A444FF0000C10F8D9
:10313000013B13F0070408BF10F8014B1D1108BF35
:1031400010F8015B641E05D010F8016B641E01F8D5
:10315000016BF9D113F0080F1EBF10F8014BAD1C25
:103160000C1B09D16D1E58BF01F801CBFAD505E043
:1031700014F8016B01F8016B6D1EF9D59142D6D39D
:10318000704700000023002400250026103A28BFC5
:1031900078C1FBD8520728BF30C148BF0B607047C9
:1031A0001FB51FBD10B510BD00F070F91146FFF737
:1031B000F7FF08F061F800F08EF903B4FFF7F2FFB3
:1031C00003BC00F095F90000094880470948004712
:1031D000FEE7FEE7FEE7FEE7FEE7FEE7FEE7FEE7C7
:1031E000FEE7FEE704480549054A064B7047000024
:1031F00039A60008ED300008181300201819002027
:10320000181500201815002053EA020C00F0698000
:103210002DE9F04B4FF00006002B1FBFB3FA83F5EA
:1032200003FA05F424FA05F65E4012BF1643B2FA1B
:1032300082F502FA05F4C5F120051EBF22FA05FC4D
:1032400044EA0C04203556EA044C4FEA144418BFF3
:10325000641C4FF000084FF00009904271EB030C22
:1032600039D3002919BFB1FA81F701FA07F6B0FA8C
:1032700080F700FA07F6C7F120071EBF20FA07FC07
:1032800046EA0C062037B6FBF4FCA7EB0507103F17
:1032900007F01F0BCBF120060CFA0BFB2CFA06F6FD
:1032A00044BFB3460026202FA4BF5E464FF0000B5C
:1032B0005BEA060C08BF4FF0010B19EB0B09ABFBE7
:1032C000027C48EB0608C01B06FB02CC0BFB03CCC0
:1032D00071EB0C01C1E70B46024641464846BDE88A
:1032E000F08B13B54FF000004FF00001AFF30080FA
:1032F000BDE81C407047032A40F2308010F0030CF8
:1033000000F0158011F8013BBCF1020F624498BF38
:1033100011F801CB00F8013B38BF11F8013BA2F1D5
:10332000040298BF00F801CB38BF00F8013B11F050
:10333000030300F05280083AC0F0088051F8043BC3
:10334000083A51F804CBA0E80810F5E7121D5CBF5D
:1033500051F8043B40F8043BAFF30080D20724BF90
:1033600011F8013B11F801CB48BF11F8012B24BF24
:1033700000F8013B00F801CB48BF00F8012B704773
:1033800002F0FF0343EA032242EA024200F002B8DD
:103390004FF000020429C0F0128010F0030C00F07E
:1033A0005080CCF1040CBCF1020F18BF00F8012BC7
:1033B000A8BF20F8022BA1EB0C0100F042B85FEA95
:1033C000C17C24BF00F8012B00F8012B48BF00F896
:1033D000012B704770477047704710B5203AC0F016
:1033E0000B80B1E81850203AA0E81850B1E8185006
:1033F000A0E81850BFF4F5AF5FEA027C24BFB1E843
:103400001850A0E8185044BF18C918C0BDE81040B3
:103410005FEA827C24BF51F8043B40F8043B08BFBC
:103420007047D20728BF31F8023B48BF11F8012B83
:1034300028BF20F8023B48BF00F8012B70474FF02F
:10344000000200B5134694469646203922BFA0E8F4
:103450000C50A0E80C50B1F12001BFF4F7AF090700
:1034600028BFA0E80C5048BF0CC05DF804EB8900F1
:1034700028BF40F8042B08BF704748BF20F8022B34
:1034800011F0804F18BF00F8012B7047754600F00F
:103490002BF8AE4605006946534620F007008546E6
:1034A00018B020B5FFF79EFEBDE820404FF00006A3
:1034B0004FF000074FF000084FF0000B21F007011C
:1034C000AC46ACE8C009ACE8C009ACE8C009ACE85F
:1034D000C0098D46704710B50446AFF30080204602
:1034E000BDE81040FFF769BE00487047B4120020E5
:1034F00001491820ABBEFEE726000200704700001D
:1035000004480168490704D56FF00401016005F023
:10351000F8BD70470024014070B5114C02212046CF
:1035200000F024F802210F4800F020F8022000F0FB
:10353000B5FD0021204600F01AF90B4D0021284668
:1035400000F0B8FD084A0421083AD160012128465C
:1035500000F0B0FD2046BDE87040012100F007B941
:10356000002401400028014008000240C9430160D6
:1035700070470029816802D041F0010101E021F08B
:103580000101816070470029816802D041F4807197
:1035900001E021F480718160704700000D4910B591
:1035A000884202D1012144150AE00B49884202D128
:1035B0000121041504E0094988420AD10121CC0304
:1035C000204606F07DFD2046BDE81040002106F0B3
:1035D00077BD10BD0024014000280140003C01409F
:1035E0000029816802D041F4801101E021F48011AA
:1035F000816070470029816802D041F4004101E0F8
:1036000021F4004181607047826822F4E0420A435D
:103610008168914200D0826070470146002089682D
:10362000490700D5012070470246002012680A426F
:1036300000D00120704708B5084428300090006889
:1036400080B208BD002A4268C9B201D00A4300E036
:103650008A4342607047000010B542680E4B0C79F7
:103660001A400B6842EA04221343436082680B4B02
:103670001A40D1E9024323434C7942EA44021343FE
:103680008360C26A097C22F47002491EC9B242EA10
:103690000151C16210BD0000FFFEF0FFFDF7F1FF18
:1036A00070B5072609290AD9C568A1F10A0404EBF7
:1036B0004404A640B543A3401D43C56007E0056927
:1036C00001EB4104A640B543A3401D430561836B54
:1036D000C3F30154121B921C02EB82021F2494407C
:1036E000A34391400B43836370BD826B491E22F458
:1036F000401242EA01518163704770B507260929DB
:103700000AD9C568A1F10A0404EB4404A640B543F4
:10371000A3401D43C56007E0056901EB4104A640D5
:10372000B543A3401D4305611F23072A09D2446BFB
:10373000521E02EB820293409C4391400C4344632F
:1037400070BD0D2A09D2046BD21F02EB8202934096
:103750009C4391400C43046370BDC46A0D3A02EB74
:10376000820293409C4391400C43C46270BD002987
:10377000816802D041F4A00101E021F4A001816040
:1037800070470029816802D041F4021101E021F460
:10379000021181607047816841F0040181607047C7
:1037A00000210160017141718160C16001210174DA
:1037B0007047000070B5194A194C9088A18868B10B
:1037C000D38819448DB2174909780023012907D0FD
:1037D0005178142905D2491C517002E0918016E0FD
:1037E0005370854202D900F101000FE00FD20B485F
:1037F000517880881429A0F1010080B206D2117896
:10380000491CC9B21170052901D3137090809088AA
:1038100007F06EFE08F054FBE07070BD78000020E9
:103820006404002065020020F0B50F4D0F4C00210C
:103830006E88AF8DA378084604F11402BE4201D908
:1038400022F8136032F81060401CC0B231441028D6
:10385000F8D30809A8805B1CD8B2A070102801D347
:103860000020A070F0BD00001C040020900000208B
:10387000FEE70000F0B55E4944F278530C228878E8
:1038800038B301283ED045F20C1346F61044032805
:1038900051D045F6A04545F2E84646F2584705287E
:1038A00060D048F6F12C042871D006286ED00E8125
:1038B00046F6FE5048818C81CB8144F61E7008820A
:1038C0004D8241F2CC00888240F66E70C882494831
:1038D0002EE043F22C20088144F6541048818B815D
:1038E00042F29860C88142F2AA40088242F65060D3
:1038F000488240F6980088824FF4FA60C8823D48BA
:10390000903815E00B8145F6B220488145F6C40099
:10391000888143F6E410C88143F2F67008824B8236
:103920004FF44860888240F61C40C88231486038B5
:1039300088610A77F0BD0B814C8146F6340088819E
:1039400044F64230C88144F26670088245F2FA209B
:10395000488241F20400888240F63C70C8822548C3
:103960003038E5E70D814FF4F740488147F6921073
:103970008881CE810B824F8241F25C20888241F2A5
:103980003010C8821B483030D2E700E015E00C81CF
:10399000A1F80AC048F603108881CF8146F27C0066
:1039A000088247F2C830488241F27C50888241F256
:1039B0005040C8820F486030BAE748F23930088179
:1039C0004AF2192048814AF22B00888147F2A470FC
:1039D000C88147F2B6500882A1F812C041F6902083
:1039E000888241F63800C88202489030A0E7000083
:1039F0006404002032C4000830B54FF480742502FE
:103A00000822102340292ED010DC072925D007DCFE
:103A1000042924D005291DD0062900D1846030BD99
:103A200008291ED02029FAD1026130BDB1F5806F7E
:103A30001FD008DCA14218D0B1F5007FF5D1816913
:103A400021F0020118E0A94218D0B1F5003FECD1F5
:103A5000436030BD0121816030BD856030BDC260F2
:103A600030BDC36030BD036130BD816921F001010B
:103A700002E0816921F00401816130BD426030BD06
:103A8000094910B588424FF0010101D14C0601E00F
:103A90004FF08064204606F0FBFA2046BDE8104057
:103AA000002106F0F5BA000000640040202209B1B0
:103AB00002617047C2607047F0B5827A2F4D0121D4
:103AC00091402A6842F001022A602C4E1C3632686E
:103AD0008A433260294A047B294B0C32A4B914680A
:103AE0008C4314604488C78844EA0744877A03EB10
:103AF000C707C7F840460488878844EA0744877A9E
:103B000003EBC707C7F84446047B012C12D11468A5
:103B10000C431460847A026803EBC4044FEA324217
:103B2000C4F84026847A426803EBC4034FEA324269
:103B3000C3F84426114AC37A121D002B136806D01D
:103B40000B4313600D4A0389143213B104E08B4315
:103B5000F7E713688B4313600389012B02D11368C5
:103B60000B431360407B012802D13068084330606A
:103B7000286820F001002860F0BD000000660040C9
:103B800000600040002A426901D00A4300E08A43F5
:103B90004261704710B50368002223F002030360FE
:103BA000036843F0010303604FF6FF7300E0521C0B
:103BB0004468E40701D19A42F9D14268D2073ED065
:103BC0008A79012A02683CD022F080020260CA7918
:103BD000012A026838D022F0400202600A7A012AE3
:103BE000026834D022F0200202604A7A012A026878
:103BF00030D022F0100202608A7A012A02682CD0AA
:103C000022F008020260CA7A012A026828D022F053
:103C1000040202608A78CC78920742EA04620C7946
:103C200042EA04424C79098842EA0452491E0A4396
:103C3000C261016821F001010160002114E000204F
:103C400010BD42F08002C1E742F04002C5E742F0F9
:103C50002002C9E742F01002CDE742F00802D1E7A6
:103C600042F00402D5E7491C4268D20701D09942CC
:103C7000F9D14068C007E2D1012010BD10B400EBBB
:103C80000113D3F8B04114F004041472D3F8B04116
:103C900030D0E4085460D3F8B04104F00204547208
:103CA000D3F8B44104F00F049472D3F8B441240A59
:103CB000D474D3F8B841D472D3F8B841240A147339
:103CC000D3F8B841240C5473D3F8B841240E94733C
:103CD000D3F8BC41D473D3F8BC41240A1474D3F88C
:103CE000BC41240C5474D3F8BC311B0E937410BC2B
:103CF000FFF7DCBE640D1460CDE730B5024600204E
:103D000093685B0108D49068000101D5012003E0AD
:103D10009068C00037D5022002EB0012D2F8803143
:103D200003F00103C2F880310B7A73B3D2F88041FB
:103D30004D681C434B7A43EAC5031C43C2F88041DB
:103D40008B7A03F00F038B72D2F8843123F00F03C8
:103D5000C2F88431D2F884318C7A2343C2F884319A
:103D6000CB7ACC6843EA0423C2F88831CB7B09695B
:103D700043EA0121C2F88C11D2F8801141F001010F
:103D8000C2F8801130BD042030BDD2F880314C7AA9
:103D900023430C8843EA4453C2F88031D0E7000043
:103DA0002DE9F0411B4F1C491C4C7878B1FBF0F019
:103DB000B4F9161048430014E08108BF4FF6FF70B5
:103DC0001DD007F030FE06460D46B7F9060007F095
:103DD0002AFE6FF0060208F01AFA0022104B07F0D4
:103DE0004DFE32462B4607F069FC00220D4B07F0D2
:103DF00045FE00220C4B07F061FC07F0E7FD208137
:103E0000E18880B288422CBF401A00206081BDE862
:103E1000F08100004C04002000A60E001C040020CD
:103E2000004CED4000004940000059401248818A92
:103E3000322998BF002206D94289B2F5007F88BF97
:103E40004FF4007200D942810C4A927892003C29CA
:103E500098BF101D0CD9642998BF02F1080007D93A
:103E60004089202828BF202002D2082898BF082097
:103E700003490881704700001C04002090040020C2
:103E800070030020F8B55448544A4FF44871858AAD
:103E900010684FF47A7E4843B0FBFEF15048008929
:103EA00000EBC00303EB001301EBC3011160B1FB96
:103EB000FEF18AB200B900224A484C4C0A23817AAA
:103EC00049484D4F80F89710A188B1FBF3F6B1FB3C
:103ED000F3F180F89860464E090A367801EB8601C6
:103EE000667F01EBC60606EB851180F89910A908DC
:103EF00080F89A103F490E7A80F89B6080F89C20E9
:103F0000002680F89D6080F89E6080F89F6080F8B1
:103F1000A060A0F89520E288A0F84A20FA886424DE
:103F2000B2FBF4FCB2FBF4F2A0F848C07F88A0F822
:103F3000D070A0F8BC20314AA0F8C0509588B5FBDD
:103F4000F4F4240694FBF3F3C0F8C8309279120617
:103F500092FBFEF2C0F8CC20294A90F8A230937070
:103F60000246B0F8B44092F8A1200CB9DB0701D0AA
:103F7000092305E012F00F0304D0FF2404EB4303F0
:103F80004B7000E04E7054090B78120964F345132E
:103F900062F341030B70C3F34011A0F8C610808D8B
:103FA000202818D11748017811B10078032812D1C0
:103FB00040F20110ADF8000001226946124806F0F7
:103FC0003BF912480168124A01F4E06111430160B3
:103FD000BFF34F8FFEE7F8BD1C040020380000201F
:103FE00090030020840400208C0200206404002040
:103FF0002200002090040020F6030020C4030020CB
:104000007003002065020020002800080CED00E08D
:104010000400FA05174810B5026941680A231144E3
:10402000B1FBF3F414494C6304682244B2FBF3F28D
:104030008A6382684A64C28ACA63104C008B08642F
:10404000E089A8B1B0F5807F12D00220088091F8F5
:10405000A50080070BD1E078C00608D403F00AF968
:1040600007490120C870E07840F01000E07010BDF2
:104070000020EBE79C0400208C020020700300204D
:104080002800002010B5022000F08EF8002802D091
:1040900001490720486010BD00000240C10002D560
:1040A00002490860704702494860704704040240B2
:1040B000000002400029016802D041F0010101E046
:1040C00021F0010101607047016821F001010160E8
:1040D0000021016041608160C1603149304A083986
:1040E000904203D1486840F00F0006E02C4A143299
:1040F000904204D1486840F0F00048607047284A78
:104100002832904203D1486840F47060F5E7244AB1
:104110003C32904203D1486840F47040EDE7204AB9
:104120005032904203D1486840F47020E5E71C4AC1
:104130006432904203D1486840F47000DDE7184AC9
:104140007832904203D1486840F07060D5E7154A54
:10415000111F904203D1086840F00F0006E0114A99
:104160001432904204D1086840F0F00008607047B3
:104170000C4A2832904203D1086840F47060F5E799
:10418000084A3C32904203D1086840F47040EDE7A1
:10419000044A50329042EAD1086840F47020E5E7C2
:1041A000080002400804024002460020D10001D568
:1041B000034900E003490968114200D0012070471B
:1041C000000402400000024030B5026847F6F07378
:1041D0009A430C6A8B682343D1E904452C4323435B
:1041E0008C692343CC6923434C6A23438C6A234361
:1041F00013430360CA6842600A6882604968C1600C
:1042000030BD704730B5044600234FF47A7504E0A2
:10421000284600F005F85B1C9BB2A342F8D330BDE2
:10422000002206E00021491C89B20F29FBD3521C51
:1042300092B28242F6D370472DE9F04102F06EFD52
:104240008C4C012100256076227E002A2DD0A37E91
:1042500000F0040703F00408DFF81CC20222874EB6
:1042600047455BD1BCF90070B7F57A7F56DDB4F8ED
:104270004E70B7F57A6F28BF22740BD2B7F5FA6F7C
:1042800005D994F81080B8F1000F08BF21747F1C85
:10429000A4F84E70E77E002F1FBFA77C002F677C1D
:1042A000042F0ED0277F2FB10BE0A076E576217684
:1042B000BDE8F081677F002F1FBFA77F002F042775
:1042C000677400F0020803F00207B84567D1BCF933
:1042D0000070B7F57A7F62DDB4F85070B7F57A6F89
:1042E00028BF22740BD2B7F5FA6F05D994F8108065
:1042F000B8F1000F08BF21747F1CA4F85070E77E4E
:10430000002F1CBFA77C002F19D0677C022F1CBF79
:10431000277F002F13D0677F6FB110E0B6F91670BA
:10432000322FC8BF2574A4F84E502177677C042F24
:1043300008BF6574C5E7A77F002F18BF6274C70761
:10434000B7EBC37F38D1BCF90030B3F57A7F33DDEA
:10435000B4F85230B3F57A6F28BF227409D2B3F59E
:10436000FA6F03D9227C002A08BF21745A1CA4F8D2
:104370005220E27E002A1CBFA27C002A0BD0627C65
:10438000012A1FBF227F002A627F002A03D0A27F5A
:10439000002A08BF6174A076E07EF8B919E0B6F98A
:1043A0001670322FC8BF2574A4F850506177677C0F
:1043B000022F08BF6574C2E7B6F91620322AC8BFBB
:1043C0002574A4F85250A177617C012908BF657457
:1043D000E1E7A07C10B125776577A577A07C284F11
:1043E000E076387801281CBFB6F916000A28A8BF65
:1043F000BDE8F08102F00CFCA4F84E50A4F8505037
:10440000A4F85250B18A322988BFBDE8F0811D4915
:104410004988B1F5BA5F88BFBDE8F0811A490989BA
:10442000002918BFBDE8F0811849CA7812F0010FC1
:1044300006BF0A7C002ABDE8F0813A78032A1EBF35
:104440003A78002ABDE8F081A27C002A1ABFE27EF9
:10445000002ABDE8F081002814BF0728BDE8F081DC
:10446000A574C88930F00400C88108BF3D70BDE85C
:10447000F081000094010020660200201C0400204E
:1044800065020020C4030020900300207003002078
:10449000154810B50121A0F8A910052180F8AB102E
:1044A0002D2141864FF4A071018640F23A71C185F9
:1044B000002180F8A11018220CA10A30FEF71BFF82
:1044C0000948152210A15330FEF715FF06481522A2
:1044D0000DA16830FEF70FFF03481822BDE8104019
:1044E00002A17D30FEF707BF8C020020556E6B6E77
:1044F0006F776E20202020202020202020202020C8
:104500002020202000000000556E6B6E6F776E201B
:1045100020202020202020202020202020000000FB
:10452000194810B519494288A1F8A920027981F8E3
:10453000AB20C2884A8602890A864289CA85027BE4
:1045400081F8A120807B81F8A2000F490F48182232
:1045500010310A30FEF7CFFE0B490C4815222831E6
:104560005330FEF7C8FE0849084815223E3168302E
:10457000FEF7C1FE0449054818225431BDE8104039
:104580007D30FEF7B8BE0000401000208C020020F5
:1045900070B5234D06200024288022481822B0F848
:1045A000A910698090F8AB10A980418EE980018E36
:1045B0002981C18D698190F8A110A98190F8A2008C
:1045C0001849E8810A3105F11000FEF794FE1549FB
:1045D0001522533105F12800FEF78DFE11491522F1
:1045E000683105F13E00FEF786FE0E4918227D3146
:1045F00005F15400FEF77FFE002035F81010401C36
:10460000214480B28CB26328F7D3A5F8C640642257
:104610000349054805F010FE04490020C87070BD2C
:10462000401000208C02002000EC00082800002030
:1046300070B5194C207801282CD1002006F036F8EE
:1046400000F04CF9154D284600F0ECF804281BD179
:1046500013480188284600F023F912480188A81C55
:1046600000F01EF910480188281D00F019F90F48C4
:10467000807B000602D445F2757101E04FF6FF71B0
:104680000648801D00F00CF900202070BDE8704045
:1046900000F0FEB870BD00008401002000F00008AA
:1046A0008C0100208E01002090010020700300206A
:1046B0002DE9F041134E3078002821D072B6002049
:1046C00005F0F4FF00F00AF90F4D284600F0AAF8B3
:1046D0000027042810D10D4CDFF8348067806088F3
:1046E00038F8101005EB400000F0DAF86088401C44
:1046F00080B260800728F2D3377000F0C9F862B644
:10470000BDE8F081A001002000F400084600002070
:10471000A81100202DE9F041DFF86C8098F8000026
:1047200000282ED072B6002005F0C0FF00F0D6F8A9
:10473000164F384600F076F8002604281CD114489D
:10474000144D164C0068010C2980688012480078CE
:10475000A880EE802E816889401C6881A680A08890
:1047600035F8101007EB400000F09AF8A088401CC4
:1047700080B2A0800628F2D388F8006000F088F8A4
:1047800062B6BDE8F08100009F01002000F800083B
:1047900004020020B6110020A101002046000020E4
:1047A00030B517490888174A10804888164A108083
:1047B0008888164A1080C888154A0023164C108035
:1047C000144A1380108801EB4005B5F8005424F812
:1047D0001050401C80B210800728F3D30F4C138078
:1047E000108801EB4005B5F8005824F81050401C23
:1047F00080B210800628F3D30948037030BD000052
:1048000000F000088C0100208E01002090010020A3
:104810009201002046000020A8110020B6110020BF
:104820008401002070B50E4E0546304600F062F857
:10483000042813D10B4C206940F00200206165610F
:10484000206940F040002061304600F053F8052810
:1048500004D0216941F6FD721140216170BD000054
:10486000FFFF0F000020024008490420CA68D20759
:1048700001D001207047CA68520701D50220704755
:10488000C968C906FBD5032070470000002002401C
:104890000248016941F08001016170470020024037
:1048A000F0B506464FF6FF770D46384600F022F881
:1048B00004280FD1084C206940F0010020613580A8
:1048C000384600F017F8052804D0216941F6FE7239
:1048D00011402161F0BD0000002002400348024960
:1048E0004160034941607047230167450020024051
:1048F000AB89EFCD00B50346FFF7B6FF02E0FFF747
:10490000B3FF5B1E012803D0002B00D1052000BDA2
:10491000002BF4D1FAE700002DE9F04100244FF418
:10492000C878254642465A495A4805F079FC584805
:104930004FF4C77630F81410641C2944A4B28DB229
:10494000B442F7D901880124534F0C2903D1B0F8A0
:104950001E03A84210D0FFF7C1FF5048FFF762FFC7
:104960004F48FFF75FFF4F48FFF75CFFFFF790FFEF
:1049700005F0ECF83C7001E005F090F900254246A6
:1049800049494A4805F04CFC4749002031F81020BD
:10499000401C2A4480B295B2B042F7D908880C284E
:1049A00003D1B1F81E03A84203D000F009FB7C70CC
:1049B0000BE014223E48891CFEF79DFC3A493C4816
:1049C000142216311430FEF796FC002514223949C2
:1049D000394805F025FC3749002031F81020401CEB
:1049E0002A4480B295B21328F7D30A8833480026A8
:1049F000092A02D1CA8CAA4205D046600660068305
:104A00008660BC7012E08A884B8802EB03424260E9
:104A10000A89CB8802EB034202608A894B8902EB48
:104A200003428260C989018302F024FC21490025E8
:104A300064222831224805F0F3FB1E49002028316A
:104A400031F81020401C2A4480B295B26328F7D375
:104A50000888062803D1B1F8C600A84203D0FFF7A2
:104A600017FDFC7001E0FFF75BFD164940F2714352
:104A7000B1F90620487842435A438A6000044FF453
:104A80007A52B0FBF2F0C8600F480680BDE8F081B2
:104A9000D809002000E000082800002000F00008ED
:104AA00000F4000800F80008F80C002000E40008FA
:104AB000B80400201810002000E800089C04002022
:104AC00000EC00084C040020140000201B4810B526
:104AD000017811B1007803282FD11948C07848B166
:104AE00018480168184A01F4E06111430160BFF3FE
:104AF0004F8FFEE71548017819B1BDE8104005F069
:104B000085B9417819B1BDE8104000F09FBA8178AD
:104B100019B1BDE8104004F003BFC07818B1BDE87A
:104B20001040FFF735BD0A480078002805D0FFF790
:104B3000BFFDBDE81040FFF7EDBD10BD65020020D0
:104B4000900400200CED00E00400FA05280000208D
:104B500099010020F0B5CC78002204F00F03E406A0
:104B600001D58C7823430C784FF00F0C14F0FF0F15
:104B70004FF0010E1BD005680E880EFA02F4264095
:104B8000A64210D196000CFA06F725EA070703FAA9
:104B900006F5CE783D43282E02D0482E02D002E002
:104BA000446100E00461521C082AE5D305600A88CC
:104BB000FF2A1CD94468002202F108060EFA06F505
:104BC0000E882E40AE420ED196000CFA06F7BC437A
:104BD00003FA06F7CE783C43282E00D14561CE7803
:104BE000482E00D10561521C082AE5D34460F0BD6F
:104BF00041F480328261816182618169806970479C
:104C0000F0B5144C002801DAE36900E06368450D53
:104C10002E0185B2C0F30157B540C0F30342032F04
:104C200005D0C6020AD503269640B34307E023F019
:104C30007062636823F07063636002E0AB4343F02B
:104C4000706201B12A43002801DAE261F0BD6260BE
:104C5000F0BD0000000001400246002092680A42B8
:104C600000D0012070474FF6FF7101800221817052
:104C70000421C17070470AB10161704741617047FA
:104C80002DE9F003254F264DA7F16006D7F80090D7
:104C9000288CC9F34E0195F80080091A002226F8E5
:104CA0001810B6F90010B6F902C030465FF00703DD
:104CB00030F9044F6144B0F902C022445B1EF7D1C1
:104CC0008818B6F91E10084408F10101C9B229700C
:104CD000102924BF00212970B968124B0A0DDFF892
:104CE00048C09A827A680830530CACF80030C1F39F
:104CF0004E030E4900118B80BB89C3F34E03CB805A
:104D00000B4908800B49C2F34E0008800A494FEA5C
:104D100059400880BDE8F00370470000681100208A
:104D2000CC00002070030020F60300201A000020B1
:104D30008404002064040020C40300202DE9F04115
:104D40004FF00108264F274E4446787D0025002865
:104D50004FF0400130462FD0FFF77EFF45EA400577
:104D600080213046FFF778FF05434FF480713046CD
:104D7000FFF772FF45EA8000C1B200291CBF072976
:104D8000BDE8F08104F10100C4B2042CDDD300249D
:104D9000204605F08BFC1448C470817C002908BFB4
:104DA00080F812801148C18941F00401C181104985
:104DB00003200870BDE8F081FFF74EFF45EA40058B
:104DC00080213046FFF748FF45EA8000C5B24FF426
:104DD00080713046FFF740FF40EA0501CDE7000053
:104DE0004C040020000C01409401002070030020BE
:104DF0006502002010B5234B2349B3F92E00B1F909
:104E00000620904200DAC880B3F93020B1F90610CC
:104E10008A420EDB501A80B231B1202800D92020FE
:104E2000824203DD101A02E08020F9E70020188694
:104E300010BD1648B0F90000824200DA1886144A04
:104E4000948A502C02D9B0F5FA6F04DA11488078B0
:104E50008000001D07E05089202801D9202002E0B1
:104E6000082800D20820B3F930404FF4C8729442A9
:104E700000DA1A86B3F9302010448842D7DB19864D
:104E800010BD0000C40300205A000020680200206A
:104E90001C04002090040020F0B52C4E2D4A2C4B11
:104EA000B6F8B210108800244FF4BA5544F6903783
:104EB00039B9B6F8B41021B19988A94204D29D80BD
:104EC00004E09C80508006E0B94203D2998801F545
:104ED0007A71998051805188B94200D357806421FA
:104EE00041434FF4F877B1FBF7F191806421A0F5CD
:104EF000BA50484343F2504190FBF1F0C0B2907178
:104F0000642801D964209071B6F8C400124EC0B96B
:104F10005088A84215D99D789DB9957B8DB10F4DCC
:104F2000ED78ED060DD4B2F92E20A0F5BA5050431D
:104F3000B0FBF1F0D8807078002801D07470347024
:104F4000F0BDDC8001207070F0BD00008C020020FC
:104F50005A000020C403002022000020700300201B
:104F6000FEE710B545F2555000F024F8022000F09D
:104F700015F8BDE810407F2000F016B802494CF645
:104F8000CC400860704700000030004002494AF6FB
:104F9000AA200860704700000030004001494860C6
:104FA00070470000003000400149886070470000F1
:104FB00000300040014908607047000000300040A8
:104FC00070B5142214A11A48FEF795F91848142256
:104FD00018A11438FEF78FF91548342514383524F4
:104FE00005704470312282703021C1703223037108
:104FF00041718171C27101723926467233268672FF
:10500000C3720173457338218173C273047443748E
:1050100037228274C17470BD4D312D3142452D311E
:105020002020202020202020202020200000000000
:10503000CC04002020202020202020202020202000
:1050400020202020202020200000000070B5134DDB
:105050000C210024298014221149A81CFEF74BF9C9
:105060000F491422143105F11600FEF744F900210E
:105070004FF4C77035F81120491C224489B294B20C
:105080008142F7D9A5F81E434FF4C8720349054879
:1050900005F0D2F804490020487070BDF80C0020DB
:1050A000B804002000E400082800002010B5002407
:1050B00002F058F8641CA4B2642CF9D30448417B74
:1050C000012903D1C18941F48051C18110BD000083
:1050D000700300200C4910B5C88840F6AB54431E3D
:1050E0000A4AA34208D2098801EB81014900B1FBB9
:1050F000F0F01169084410611169106808440A2130
:10510000B0FBF1F0D06010BD1C0400209C04002016
:1051100070B45B485B4AB0F90C300382B0F90E10F2
:1051200003EB410151430C1444825749564A098804
:10513000128801F50041890911F4407502F5004219
:105140005249C2F38712C2F1FF0C7CD0B5F5807FC3
:105150007AD0B5F5007F03D0B5F5407F06D00DE0DD
:1051600031F81220028131F81C1006E031F81CC021
:10517000A0F808C031F8121077E04181B0F90A2098
:10518000B0F9085003FB02F104FB15116B43CE1379
:1051900004FB02323E4990F801C0D31301F1200212
:1051A00021F81C6022F81C30B1F90030B1F902502E
:1051B000B2F900401D44B2F902302344B1F9044071
:1051C000B1F906102C44B2F904502144B2F906207A
:1051D000891C2B4489101A44C183911C0CF10102D3
:1051E00041F38F01D2B281824270042A04BF0022AF
:1051F00042704A422749B1F9003003FB02F4B1F989
:1052000004305A434B694FEAE37C9B184CEBE27243
:10521000D1F810C04FEAEC75BCEB0306954109DBF1
:10522000D1F80CC04FEAEC75B3EB0C06AA41A8BF4D
:105230004B6101DAC1F814C04A69B1F90A3022445D
:10524000D213934201E00AE011E0AABFB1F90810BD
:105250001A469142C8BF0A46428370BC704731F873
:1052600012205242028131F81C10494285E731F880
:105270001CC0CCF1000CA0F808C031F812107CE77B
:10528000CC000020326CFFFFF4010020F4C40008C1
:1052900028110020F80400202DE9F041324C0121B2
:1052A00000256078314ECF0370B1012840D002282C
:1052B00008D1A078401CC0B2A070032802D3A5700A
:1052C000E5706570BDE8F08129480078012811D0AB
:1052D000284A0020D28901FA00F31A420ED0A570A4
:1052E0002571401CE0706170002239463046FFF79E
:1052F000C2FC07E000223946304615E0401CC0B22F
:105300001028E8D3E0780028DCD1A078401CC0B297
:10531000A0700228D6D3A570B1683046090401D523
:10532000002200E001223946BDE8F041FFF7A3BCAE
:105330002079401C2071B068000401D5002200E0F3
:10534000012239463046FFF796FCE078217940008B
:10535000801C8842B6D2A570002239463046FFF73D
:105360008AFC02206070ADE784000020001001403C
:1053700065020020700300203149B1F90220B1F923
:1053800004C0624508BF70472E484378012B18BF00
:10539000704730B42C4B9C8A782C2AD82B4B5C78E5
:1053A00014F0040F1DBF1B79002B04230823C488AD
:1053B00004F10104A4B2C4809C429CBF30BC70477D
:1053C0000023C38002F120041D4840F667036445B2
:1053D000B0F9000016DA1E4D2D88242D12D222B20B
:1053E0004A808242B2BF984230BC7047488030BC8D
:1053F00070475D89174B184C0A2D5B78E35C88BFBA
:105400005B08D4E702F11004644507DA22B24A804F
:105410008242B2BF984230BC7047E7E70CF12003EC
:105420009A42DEBFA1F802C030BC7047203A12B2E7
:105430004A808242C8BFEF28D8DC30BC70470000E9
:1054400084040020640200201C040020700300205B
:10545000BA01002090040020FCCB00080848007826
:10546000002808BF70470748007B002818BF704716
:105470000020054948610549486105490880704791
:105480009901002070030020F8040020E0040020AF
:10549000E6000020094910B500204861084948612C
:1054A0000849088000F0A0FD0748C08A002818BFFE
:1054B00010BDBDE8104000F089BD0000F8040020D8
:1054C000E0040020E60000201C04002070B5324CEF
:1054D000207800281CBF2078032807D12F494FF0DF
:1054E000EF0048804FF0000005F0E0F8217800223E
:1054F0002B48012948D02B49B1F916300A2B43DA41
:10550000898A322940D228494988B1F5BA5F3BD20D
:1055100026490989002901BFC17811F0010F017CDA
:10552000002931D1C18911F0080F04D0204B1A7025
:1055300021F00801C1818BB21E4913F0400F08D041
:10554000B1F800C00D89AC4503D94A7723F0400378
:10555000C3819BB213F4006F09D0DFF85CC0BCF8C4
:105560000AC0BCF1040F3CBF23F40063C3819BB2AB
:1055700013F0200F08D0B1F800C08D89654503D91C
:105580008A7723F02001C1812178032902BFC089D5
:105590000028227070BD00006502002084040020F5
:1055A000700300201C040020C4030020900300208E
:1055B000A401002064040020900400202DE9F04F95
:1055C000DFF838C48EB00022BCF90060BCF90230AC
:1055D0000193F31A114610460D9348BF5B42DFF862
:1055E0001CC4019CBCF904C0B4EB0C0CCDF828C061
:1055F0004CBFA3EB0C036344102BB4BF1023B3F5D3
:10560000006FC8BF4FF40063FD4CB4F90070B4F9EB
:1056100002C0CDF800C0B7EB0C0CCDF830C048BFCD
:10562000CCF1000CF64C009DB4F904402C1B0994FD
:105630004CBFACEB040CA444BCF1100FB4BF4FF052
:10564000100CBCF5006FC8BF4FF4006CDFF8B483DA
:10565000B8F90050B8F90290B5EB09040B9448BFB3
:105660006442DFF8A083B8F90480B9EB0808CDF8EC
:1056700020804CBFA4EB08044444102CB4BF102479
:10568000B4F5006FC8BF4FF40064DFF87C8398F86E
:1056900003A0BAF1000F14BF4FF0010B4FF0000B45
:1056A00088F804B0DFF8608398F807B0B8F826E00F
:1056B000CDF81CE0B8F824E0CDF818E008F13A0E77
:1056C000BBF1070FBEF900E00EEB4E0ECDF814E073
:1056D000B8F82280CDF81080DFF82083B8F9008078
:1056E00008EB4808CDF80C80DFF81883B8F9008083
:1056F00008EB4808CDF80880DFF8108380F01C83A1
:10570000DFE80BF0FE0483FDFCFBFA00C0480168F3
:105710000798BD4A401A10F5804FB4BF4046B0F517
:10572000804FC8BF4FF48040411BA142C8BF281919
:1057300004DCC4F1000B8B45C8BF281B1063BAF111
:10574000000F1DD0B3490C680699091BCC1BB4F59A
:10575000805F02DC14F5805F01DA0024147111F51A
:10576000804FB4BF4146B1F5804FC8BF4FF4804170
:10577000CA1B62452ADCCCF10004A2422FDA2CE0DD
:10578000411B48BF49420C9A002A099A09D4002AB1
:1057900058BF39440ED5059A0A440099511A491048
:1057A00008E0002A48BF791A04D4059A521A0099D1
:1057B000511A491011F5804FB4BF4146B1F5804FE1
:1057C000C8BF4FF48041CA1B624502DD07EB0C01E4
:1057D00005E0CCF10004A24201DAA7EB0C010A18A3
:1057E000524212F5804FB4BF4246B2F5804FC8BF57
:1057F0004FF48042A2EB060C9C4500F397825C427A
:10580000A44580F2998200F096BA81480268079810
:105810007D49801A10F5804FB4BF4046B0F5804FE7
:10582000C8BF4FF48040421BA242C8BF281904DC05
:10583000C4F1000B9345C8BF281B0863BAF1000FE1
:105840001CD0744A1468049A121B941BB4F5805F30
:1058500002DC14F5805F01DA00240C7112F5804F30
:10586000B4BF4246B2F5804FC8BF4FF48042911B8F
:10587000994229DC5C42A1422CDA2AE0411B48BF54
:1058800049420D9A002A0A9A09D4002A58BF721870
:105890000ED5039A0A440199511A4A1008E0002AC9
:1058A00048BF721A04D4039A521A0199511A4A1025
:1058B00012F5804FB4BF4246B2F5804FC8BF4FF4D7
:1058C0008042911B994201DDF21803E05C42A14243
:1058D00000DAF21A1118494211F5804FB4BF41465F
:1058E000B1F5804FC8BF4FF48041CB1B63457DDCD1
:1058F000CCF10004A34204E099E113E195E003E058
:1059000012E280F219828CE04248026804983E4913
:10591000821A12F5804FB4BF4246B2F5804FC8BF1D
:105920004FF48042901B9842C8BFF21804DCC3F1C8
:10593000000B8345C8BFF21A0A63BAF1000F1CD0EE
:10594000334803680798C01A431BB3F5805F02DC35
:1059500013F5805F01DA00230B7110F5804FB4BF9F
:105960004046B0F5804FC8BF4FF48040411BA14274
:1059700029DC634299422CDA2AE0901B48BF40425E
:105980000B990029089909D4002958BF28440ED53D
:1059900002990844A0EB0900401008E0002948BF24
:1059A000281A04D40299081AA0EB0900401010F537
:1059B000804FB4BF4046B0F5804FC8BF4FF4804021
:1059C000411BA14201DD281903E06342994200DA3C
:1059D000281B1118494211F5804FB4BF4146B1F55B
:1059E000804FC8BF4FF48041CB1B00E001E063450E
:1059F00012DD07EB0C0100F09FB900000001002050
:105A0000060100200C010020CC00002000C0FFFF98
:105A10003C2801403C240140CCF10004A34280F228
:105A20008B81A7EB0C0100F087B9F7480268049955
:105A3000F6488A1A12F5804FB4BF4246B2F5804F3D
:105A4000C8BF4FF48042911B9942C8BFF21804DCD2
:105A5000C3F1000B8B45C8BFF21A0263BAF1000F05
:105A60001DD0EB490B680699C91ACB1BB3F5805FB3
:105A700002DC13F5805F01DA0023037111F5804F1A
:105A8000B4BF4146B1F5804FC8BF4FF48041C81B39
:105A900060452ADCCCF1000398422FDA2CE0901B01
:105AA00048BF40420C990029099909D4002958BFE0
:105AB00039180ED5059901440098081A411008E0DC
:105AC000002948BF391A04D40599091A0098081A00
:105AD000411011F5804FB4BF4146B1F5804FC8BFAA
:105AE0004FF48041C81B604502DD07EB0C0105E067
:105AF000CCF10003984201DAA7EB0C0150184042A8
:105B000010F5804FB4BF4046B0F5804FC8BF4FF48A
:105B10008040431BA3426EDCC4F1000C634580F25D
:105B20000B8182E0BA4802680699B848891A11F5D3
:105B3000804FB4BF4146B1F5804FC8BF4FF480419C
:105B4000CA1B6245C8BF07EB0C0105DCCCF1000B9A
:105B50009345C8BFA7EB0C010163BAF1000F22D037
:105B6000A94AD2F800C0049AA2EB0C02A2EB060CE0
:105B7000BCF5805F02DC1CF5805F03DA4FF0000C9F
:105B800080F804C012F5804FB4BF4246B2F5804F92
:105B9000C8BF4FF48042901B98422ADCC3F1000C2E
:105BA00060452EDA2CE0C81B48BF40420D9A002AFF
:105BB0000A9A09D4002A58BF32180ED5039A024413
:105BC0000198101A421008E0002A48BF321A04D483
:105BD000039A121A0198101A421012F5804FB4BF9E
:105BE0004246B2F5804FC8BF4FF48042901B9842A6
:105BF00002DDF21805E012E0C3F1000C604500DAA6
:105C0000F21A5018404210F5804FB4BF4046B0F52C
:105C1000804FC8BF4FF48040431BA34201DD2819C9
:105C20008AE0C4F1000C63457EDA281B84E07648E4
:105C300001680698754A411A11F5804FB4BF414674
:105C4000B1F5804FC8BF4FF48041C81B6045C8BF45
:105C500007EB0C0105DCCCF1000B8345C8BFA7EBBB
:105C60000C011163BAF1000F22D06948D0F800C0CE
:105C70000798A0EB0C00A0EB050CBCF5805F02DCE4
:105C80001CF5805F03DA4FF0000C82F804C010F5B9
:105C9000804FB4BF4046B0F5804FC8BF4FF480403E
:105CA000421BA2422ADCC4F1000C62452DDA2BE033
:105CB000C81B48BF40420B9A002A089A09D4002A00
:105CC00058BF28440ED5029A1044A0EB090040109A
:105CD00008E0002A48BF281A04D4029A101AA0EB40
:105CE0000900401010F5804FB4BF4046B0F5804F1A
:105CF000C8BF4FF48040421BA24201DD281904E0D6
:105D0000C4F1000C624500DA281B0A18524212F551
:105D1000804FB4BF4246B2F5804FC8BF4FF48042B7
:105D2000A2EB060C9C4500E006E001DDF21803E062
:105D30005C42A44500DAF21A364B1B78012B3ED0A8
:105D4000354900208B1D888001F10C0298809080DD
:105D5000488058805080088018803439108008634B
:105D60002D48B0F90020343800F13A018281B1F9B0
:105D70000010C181D0F830C0BCF1000FB8BFCCF129
:105D8000000C264BB3F906309C4513DC002AB8BF43
:105D900052429A420EDC0029B8BF4942994209DCBE
:105DA0001F49B1F900100029B8BF49429942D8BF34
:105DB000002100DD012181710EB0BDE8F08F164B8E
:105DC000DDF804C0A3F804C003F1060C009CACF895
:105DD000044003F10C04A4F804905E80ACF8027057
:105DE00065801A80ACF800102080A3F13400016BAC
:105DF00011F5804FB4BFC0F83080B1F5804FC4BFFB
:105E00004FF480410163ABE73C240140CC0000200B
:105E10003C2801406502002000010020840400208D
:105E20000C0100202DE9F041604C614DDFF88481C8
:105E30006078614F10F0020F4FF0010608D004F0B7
:105E4000A9F8B7F93000B5F9301088420CDD0AE046
:105E500010F0040F08D005F035F8B8F91000B5F9C6
:105E60003010884200DD267160784FF0000610F097
:105E7000010F18D0FEF7BEFF607810F0020F07D0B8
:105E8000B5F9300078B1B7F9301088420ADA0AE083
:105E900010F0040F06D0B5F9300020B1B8F9101099
:105EA000884200DB2671227C44484FF4C8734FF4CB
:105EB0007A717AB1B4F90620B2F5C87FB4BFE38035
:105EC000B2F57A7FC8BFE18046DAE18801F10201CC
:105ED000E18041E0627B0AB1E68060E0627C012AF9
:105EE00012D0E17811F0010F39D0B4F9061040F664
:105EF000B832B1F5C87FB4BFE380B1F57A7F15DC65
:105F0000E188491CE18022E0B4F90620B2F5C87F9F
:105F1000B4BFE380B2F57A7F06DCE288921C12B24D
:105F2000E280B2F57A7F36DDE18038E0244BB3F8C9
:105F300006C00CF1010C1FFA8CFCA3F806C0BCF1E2
:105F4000080F04D39142DCBF491CE180DE80B4F924
:105F500006109142C8BFE280818C01831BE0194981
:105F60000A78002A1CBF4988E18014D11649497873
:105F70000029B1D0217951B1617811F0020F0CBF25
:105F8000B8F91010B7F93010E180B98802E0298E15
:105F9000E18069890183B4F9061000299CDBC18A7C
:105FA000008BBDE8F04104F08DBA000070030020C2
:105FB000C4030020F6030020900300201C040020EE
:105FC0004C00002022000020900400200548002101
:105FD000C18401858170C1708171C1858184C16670
:105FE000704700009401002010B500F097FE0149B1
:105FF000C87710BD940100202DE9F041002600F083
:1060000007FE4B4C0025E07794F8202090427ED08C
:10601000A18F638C99429CBF617900291AD000BF7F
:106020004FF00107277194F90010002918BF617023
:1060300025704049895C814208BF27703AD03E49AB
:10604000895C81422AD1208D002804BF6079002814
:1060500021D113E094F9011094F90030994218BF4E
:10606000002BDDD1238D002B08BF0129D8D0E38C74
:10607000002B08BFB1F1FF3FD2D048E0E08C0628EA
:1060800009D9B4F8400040F28A21814203D96078EE
:10609000207001260EE0FF2020700BE0E178491C03
:1060A000C9B2E170032913D02449085C062818BF3F
:1060B00001260DD094F9000094F90110884203D014
:1060C000F0B1E57300F05CFE2078C8B196B117E03E
:1060D000E570002004F0EAFAA07C002808BFA7744D
:1060E0001748C18941F00401C18116490320087095
:1060F000E0E70CE0E57000F02FF900F05FFEA58707
:10610000E07F84F82000002E08BFBDE8F0810E4833
:1061100004F062FB0D490988A28C491C00EB024087
:106120004843E16E0844E066A584BDE8F0810000C4
:1061300094010020340200203C0200204402002090
:10614000700300206502002000080040280800407D
:106150002DE9F04F7A487949D0F868C00646C47BEB
:10616000B6F83480B6F84020DFF8D8E10023F67F97
:1061700000F1B00701252CB18179A1B1424588BF5A
:1061800083711EE017F8069040F2DC5B3EF819A020
:106190000AFB0BFADFF8B0B15BF82990BAFBF9F90A
:1061A000A0F82C9013E0C18C0F2984BFC18E9142BE
:1061B00007D9C18D491C89B2C185132908BF8571D2
:1061C00000E0C3856149B1FBFCF181856146C0F8FF
:1061D00064C0DFF86CC190F80790BCF832C0B9F128
:1061E000000F05D0B0F830904A4588BFC37104E075
:1061F000002C18BF624538BFC57190F80890B9F1FE
:10620000000F03D0624588BF037204E0002C18BF62
:10621000424538BF057290F80580DFF824C141F28D
:106220005559B8F1000FBCF954C006D1DFF82081F0
:1062300098F80080B8F1010F05D0A0F85630A0F80A
:106240002AC0837371E0DFF8F8A090F80EB0BAF8B6
:106250002A80BAF854A0BBF1000FAAEB08080FFA85
:1062600088F839D0C279002A08BF8373B0F92C307E
:10627000428F93424CDD048F9A1A92FBF4F292B251
:106280000C2A88BF0C22DC0004EB43031BB24B45F5
:10629000C8BF41F25553B8F1000FBABFC8F10004AE
:1062A00024B24446E40004EB6304641C94FBF3F35F
:1062B0009BB20C2B88BF0C23934228BF002206D22E
:1062C000D21A92B2062A84BF921F514325D2C2F13C
:1062D0000602B1FBF2F120E0C18C01299CBFA0F8BD
:1062E0005630A0F82AC00DD9B95D08EB48035B0011
:1062F0003EF81110594342F6AB235A4391FBF2F199
:10630000A0F85610002C1EBFC179002985730CE03F
:10631000104AA2FB01214FEA910140F2DC5208FB36
:1063200002F292FBF1F1A0F856100CEB0901A0F873
:106330005410B0F92C00BDE8F08F0000B0CA0B017A
:106340009401002090110020781100200000DC054D
:1063500065020020ABAAAAAA70B56C4C0025E17FAB
:1063600094F8200001F0040200F004039A420CD0DB
:10637000B4F84410B4F842000144A4F84010A4F862
:106380004400E087A4F8425022E001F0020200F04D
:1063900002039A420CD0B4F84810B4F84600014405
:1063A000A4F84010A4F84800E087A4F846500FE095
:1063B000C907B1EBC07F0BD0B4F84C10B4F84A0059
:1063C0000144A4F84010A4F84C00E087A4F84A5017
:1063D000A08F40086084802884BF80206084E07B98
:1063E000012118B9E08C072888BFE17394F90000F7
:1063F000002808DDE08C4FF6FF7188424FD2E08C18
:10640000401CE0844BE04ADAA571E585208DFF2829
:1064100002D2208D401C2085607A012808BF657259
:10642000A07A012808BFA572208D172837D9B4F8A3
:106430004000B0F5A07F32D2354841F67052B0F935
:10644000000090422BDD3148667BD0E922C3D0F8B2
:106450008020D0F88400002E1FBF6573C4E92A2075
:10646000C4E928C3D4E9260201BF6173C4E9282026
:10647000C4E92AC3D4E92402C4E92C02607A0228C0
:1064800008BF6572A07A022808BFA572E07A30B909
:1064900020484089A0F57F42FE3A18BFE172E18CA6
:1064A0001D48022902D204F097F91CE004F094F987
:1064B0001A490988A28C491C00EB02404843E16E4E
:1064C000E27F01441648825C164840F822100168B9
:1064D0004268114482681144C268114402694069EB
:1064E00011440844A066A584E566E08CFF2898BFA7
:1064F00070BD2078012806BF607C002870BD00F0C8
:1065000025FBBDE8704000F08DBD00009401002027
:1065100068020020B6110020000800402808004052
:10652000440200207811002000B500F0C1F91C4899
:10653000817871B1418D828D891A09B24185B0F996
:106540005A20D317B3EBE17F15D1511A002912DD80
:1065500010E0818DB0F856201144428D114409B2EB
:106560004185B0F95820D317B3EBE17F03D1891AE5
:10657000002900DD428502790021002A18BF4171FF
:1065800007D0417B0029418D08BF4942A0F8601027
:1065900000BD01224271B0F8542042858173F0E7BA
:1065A000940100202DE9F05FB04844F6E741B04C7B
:1065B000408ADFF8C4C24143AE48616741F2555694
:1065C000028A130442785343B3FBFCF3B1FBF3FAA2
:1065D000C4F87CA0A367B0F906305A4340F2714377
:1065E0005A438260A548A0F1180E8389A0F10C05DA
:1065F000A3F57F42FF3A2BD04788B0F80090A7EB75
:1066000009029642D8BFB2F5804F21DCB0F804C031
:10661000ACEB07029642D8BFB2F5804F18DCC388B6
:10662000A3EB0C029642D8BFB2F5804F10DC028972
:10663000A2EB03084645D8BFB8F5804F08DCB0F898
:106640000A80A8EB020B5E45D8BFBBF5804F2BDD5F
:106650008B488C4A00881388C2182A8042F6AA22E6
:1066600003EB020C8444A5F802C045F2555C9C443F
:106670008444A5F804C047F6FF7C9C448444A5F8F4
:1066800006C0A3F5AA4CACF1550C84449B1A1844DF
:10669000A5F808C06881AEF102000323428020F80B
:1066A000042F5B1EFAD127E0A5F800906F80A5F8B3
:1066B00004C0EB802A81A5F80A8003884289A3EBF5
:1066C000020CAEF800C0B0F802C0ACEB0303AEF8A9
:1066D00002308388A3EB0C0CAEF804C0B0F806C0FF
:1066E000ACEB0303AEF806300089A0EB0C03AEF868
:1066F0000830101AAEF80A00634801230027B0F8EA
:106700000AC0ACF57F42FF3A0AD0B4F9622040F6E5
:10671000AA2C12EB0C0FA4BF40F6AA2C94457DDAEC
:10672000C4F870A067746373206F5A4AB1FBF0F02D
:106730004FF42021B1FBF0F121865449B1FBF0F177
:1067400061865349B1FBF0F1A1864FF40031B1FBF2
:10675000F0F1E18664214143A2FB0121CA084FF414
:106760008031B1FBF0F0B1FBF2F2C01C80B24AF60E
:10677000AB2148436287800C2087E772277300F0C3
:10678000FFFAE766A78440F2CF306084607B002880
:1067900061D0D4E92001C4E92E01D4E92201C4E981
:1067A0003001D4E9240100BFC4E93201D4E92E014B
:1067B000C4E92801D4E93001C4E92A01D4E932014D
:1067C000C4E92C01A4F85670A785A77123706370E3
:1067D000A773E77300F0A2FA2F49E077095C35F858
:1067E00011103144A4F854106185A4F85810A4F88D
:1067F0005A10A4F85C10A4F85E1084F82000274812
:106800000780001F07802648018841F001010180B0
:106810002448018841F00301018000E007E0001DE9
:106820004FF6FE710180491E0180BDE8F09F02888D
:10683000B0F802C04CEA02422267DFF86CC0A2F551
:106840001032A2F51F62624524BF184A226767749E
:106850000079607368E7D4E92201C4E92E01D4E924
:106860002001C4E93001D4E926019DE76404002039
:10687000940100204C04002000A60E00A811002066
:106880001600002014000020B6110020AAAA06005D
:106890006DDB0200898888884402002028080040B7
:1068A000000800400C08004051F80C00400D0300A7
:1068B0002A4B00B5988F40F29E7188423CBF401C25
:1068C0009887B3F8422041F2DA6082423ABF521C04
:1068D000A3F84220A3F84400B3F8462082423ABF0E
:1068E000521CA3F84620A3F84800B3F84A2082427D
:1068F0003ABF521CA3F84A20A3F84C009A8F8A4250
:106900003CBFB3F84210814207D2B3F8461081422F
:106910003CBFB3F84A1081420AD300201871D873E3
:1069200042F6B451A3F840100D49C88200F028FA8D
:10693000587918B9187A08B1987820B1B3F85A0084
:10694000A3F8580000BD987900281ABFB3F85E007C
:10695000A3F85800B3F85C00F2D000BD9401002009
:106960001C0400207448C17C012918BF704772487C
:10697000407A012818BF70472DE9F04F4FF0000C06
:106980006E4E87B0301F63466246614603244568F9
:10699000641EAC44C5692B4450F8085F29448569DE
:1069A0002A44F4D1601E0CEB010703EB020800EB54
:1069B00057040025394656F8250000FB08F0001959
:1069C00004F0F8F846F82500681CC5B2062DF1D38E
:1069D00007EB0800401C470859486E4600F14C017F
:1069E00091E80E108DE80E10C06D049050180190C3
:1069F0001844029060440390DDE903100844002528
:106A0000CDF8100036F8250039460004001904F0CE
:106A1000D1F846F82500681CC5B2052DF2D34948C7
:106A20004949008880B20880009A024494B24C80A0
:106A3000019A024495B28D80029A024496B2CE80A9
:106A4000039A024497B20F81049A02441FFA82F813
:106A5000A1F80A800C31B1F80090484504D9A0EBA8
:106A60000902B2F5B67F52DCB1F802C0644504D920
:106A7000A4EB0C02B2F5B67F49DCB1F804A0554591
:106A800004D9A5EB0A02B2F5B67F40DCB1F806B036
:106A90005E4504D9A6EB0B02B2F5B67F37DC0B8955
:106AA0009F4203D9FA1AB2F5B67F30DC4A89904585
:106AB00004D9A8EB020EBEF5B67F28DC484504D207
:106AC000A9EB0000B0F5B67F21DC644504D2ACEB45
:106AD0000400B0F5B67F1ADC554504D2AAEB0500D8
:106AE000B0F5B67F13DC5E4504D2ABEB0600B0F523
:106AF000B67F0CDC9F4203D2D81BB0F5B67F06DC14
:106B000090450BD2A2EB0800B0F5B67F06DD888970
:106B1000A0F57F42FE3A1CBF401C88810848D0E99E
:106B20000912C36A8363C0E90C120348022141724F
:106B300007B0BDE8F08F000094010020C4110020D0
:106B400078110020140000209C11002070B42C4803
:106B5000467A01462B4DB1F84030CA7F00F1B004AF
:106B60004FF0010C00219EB1467A012E07BFC67C72
:106B7000002E70BC704740F23E36B3429CBF2B786B
:106B8000012B1CBF4172C1741BD0817570BC704752
:106B9000C174B3F5027F24BF70BC70472B78012B02
:106BA00007BFA25C002A70BC7047174A41F67053B9
:106BB000B2F900209A42AEBF80F809C070BC70479D
:106BC000E3E7A25C114B53F822205409827D4C3339
:106BD00043F822404AB103EB820252F8042CB2EB94
:106BE000440F02D941728175C174817D491CC9B2BB
:106BF00081750C2908BF80F813C070BC7047000075
:106C00009401002065020020680200207811002015
:106C10002DE9F047DFF8F8900026354699F81F0077
:106C200089F8150000F07AF80446DFF8E8803A4F5A
:106C300039E000BF98F815004FF0000A00284FF027
:106C40004001384636D0FEF707F84AEA400A80216C
:106C50003846FEF701F840EA0A0A4FF480713846D8
:106C6000FDF7FAFF4AEA8000C0B2A0421BD0681CC0
:106C7000C5B2002698F81500344600284FF04001B0
:106C800038462BD0FDF7E8FF44EA4004802138461F
:106C9000FDF7E2FF04434FF480713846FDF7DCFF57
:106CA00044EA8000C4B2701CC6B2032E28D2032D61
:106CB00028D2BFE7FDF7D0FF4AEA400A80213846D4
:106CC000FDF7CAFF4AEA800000F0FF0A4FF4807126
:106CD0003846FDF7C1FF40EA0A00C6E7FDF7BCFFF2
:106CE00044EA400480213846FDF7B6FF44EA8000BC
:106CF000C4B24FF480713846FDF7AEFF0443D2E7CB
:106D0000032D01D399F815402046BDE8F087000017
:106D1000940100204C040020000C014070B516487E
:106D20000024164D407D4FF040010028284610D029
:106D3000FDF792FF44EA400480212846FDF78CFFCE
:106D40000443A9152846FDF787FF44EA8000C0B236
:106D500070BDFDF781FF44EA400480212846FDF71D
:106D60007BFF44EA8000C4B24FF480712846FDF7EF
:106D700073FF204370BD00004C040020000C014054
:106D80000C4840F2DC52B0F8401051438166818FCC
:106D90004A4309490A604A608A60CA600A614A61D6
:106DA0000021C18401858170C1708171C185818498
:106DB000C166704794010020781100202DE9F0434E
:106DC000624C0025214694F901C094F90020604FDF
:106DD000C97F41F2555840F29E7004F1B0069445C7
:106DE0003FD0E5842585A573725C37F8122002EB4D
:106DF000080304F18002A4F85630515C715C37F945
:106E00001120A4F85420B4F92AC0A3EB0C01514B73
:106E100009B2A1851B78012B18BFA58506D10029D1
:106E200012DD490009B291FBF0F0A085B4F85600DC
:106E3000A4F85400A4F85A00A4F85C00A4F85E007A
:106E4000A4F85650BDE8F083A2EB0C0109B2A1856D
:106E50000029C6BF91FBF0F0A085A585A4F85620B7
:106E6000E4E7DFF8F8903C4AA9F1A003BCF1010F78
:106E70009B8F31D0BCF1FF3F18BFBDE8F083A573F5
:106E8000E573D582E584A4F856500120A070705CAB
:106E9000334A32F81020B2FBF3F2A28519F8011040
:106EA000715C37F81110618537F8100000EB0801AC
:106EB00009B2A4F85410228D082A32BFA4F85A103F
:106EC00000F25550A4F85A00B4F85A00A4F85C0037
:106ED000A4F85E00BDE8F08340F28A2C63453CBF15
:106EE000B4F84230834214D2B4F8463083423CBFF7
:106EF000B4F84A3083420CD2207950B1B4F8400043
:106F00004FF4803303EB5003B3FBF0F000B21028D2
:106F100000DA0020D082705C37F81000A4F854002A
:106F2000FFF716F9A085E07F19F80000305C37F80C
:106F30001000A4F85A0000F6AA21A4F85C104044FE
:106F4000A4F85E00A5702585BDE8F08394010020BB
:106F50009C110020650200201C0400203402002047
:106F6000901100202DE9F0412A4E307D012806BF06
:106F7000B07A0128BDE8F0814FF0000C264B644642
:106F800003F12002604602F120014FF0100500BF1E
:106F900033F8027B6D1EBC4432F8027B3C4431F86E
:106FA000027B3844F4D105094FEA1C1124094FF43F
:106FB000803003F0FFFD1949498A4843214603F018
:106FC000F9FD45F2F4014843294603F0F3FD01467B
:106FD000706F03F0EFFD316FC1F350128B18891AF7
:106FE000984203D8884228BFBDE8F081F17A002991
:106FF00018BFBDE8F0810A494989A1F57F42FE3AF0
:1070000008BFBDE8F08130670120F0720220B07245
:10701000BDE8F08194010020F411002064040020F8
:10702000B61100202DE9F00F4848867A4849DFF86C
:1070300028C10346474CB1F90020B3F84030BCF9F1
:1070400000C041F670554FF0010800217EB1867AEC
:10705000012E07BF067D002EBDE8F00F704740F2FD
:107060003E36B3429CBF2478012C1AD114E0B2F50D
:10707000D77F0DDA427A022A0AD1B3F5027F07D20E
:107080002278012A04D1AC45A4BF80F80A80C175DA
:107090000175BDE8F00F70476545D8BFB2F5577F61
:1070A00005DD8172C1750175BDE8F00F70472B4F8A
:1070B000C27D2B4C07F1200627F8123025881FFAD5
:1070C0008CF426F8125006F1200C07EB42072CF83E
:1070D000124037F8029C06EB420609F110077F09BF
:1070E00009EB070A36F802BCA9EB07070BF11006FB
:1070F00076090BEB0609ABEB06061FFA8AFABFB25C
:107100001FFA89F9B6B2AAB1BB4228BF9A450ED37D
:10711000B54228BFA9450AD30CEB420204F1800313
:1071200032F8022C934202D38032944202D9817207
:10713000C1750175C17D491CC9B2C175102908BF4F
:1071400080F81480BDE8F00F704700009401002023
:10715000840400206502002068020020F411002051
:107160006404002030B51448124B144D01785C7B48
:107170000022491C002C2C68C9B24FEA845409D063
:10718000002C05DA0170032901D102705A7330BD59
:10719000027030BD002CFBDB01700229F9D1D978D7
:1071A00021F00101D97006490A700270012058735C
:1071B00030BD00007003002084000020080C014056
:1071C00022000020F0B52848264F294D838AB0F9C7
:1071D00016202648FC894FF000064088E1070AD0B7
:1071E0002E70322B1DD80A2A1BDCB0F5BA5F18D2DC
:1071F00024F0010020E01B4995F802C04978BCF159
:10720000000F1BD02E70322B08D80A2A06DCB0F5EE
:10721000596F03D345F61032904203D3C80701D00B
:107220006E70F0BD6878401CC0B268700328F8D159
:107230006E70AE7024F00200F881F0BDA0F55960C8
:10724000B0F59B4F0BD9C80709D02878401CC0B2B5
:1072500028700228F1D12E700120A870F0BD2E7088
:10726000F0BD0000700300201C040020C4030020B7
:107270005A00002003480069002802D0024901207A
:10728000887070479C0400202800002010B500F092
:1072900019FDBDE8104001F007B800002DE9F047E6
:1072A000384E4FF4FA69384CB28A4A4509D3A0796E
:1072B000022802D2401CA07103E0F07840F02000C8
:1072C000F070F178314F88064FF001084FF000055B
:1072D00014D540F2D940824210D86079052802D2F4
:1072E000401C60710BE0C80609D4FFF7C3FF87F8A4
:1072F0000380F07840F01000F07000E06571B06934
:10730000B0B12349898A052912D8A168C0EB0010C1
:10731000491C00EB8000A160B1EBC00F09D3FFF75F
:10732000A9FF87F80380F07840F01000F07000E0CB
:10733000A560F078C00621D5B878F8B9F878E8B932
:10734000002003F0B3F91348057000224FF40061E8
:107350001148FDF790FCB08A48450FD9E079401CF0
:10736000C0B2E0710A280AD30C4801680C4A01F443
:10737000E06111430160BFF34F8FFEE7E571BDE8A7
:10738000F087000070030020840000202800002007
:107390001C04002065020020000C01400CED00E000
:1073A0000400FA052DE9F84FFF4F00263546B7F9DE
:1073B0001C30B7F90A20B7F91AC003FB02F1B7F97C
:1073C00008000CFB02F20CFB001103FB102041F340
:1073D000CF31F98241F24C4240F3CF30514340F675
:1073E000B832388342435042431811445B10C1F114
:1073F000000134464FEA6102009347D5002AB8BF26
:10740000052103DB0028D4BF04210321F9710021E9
:10741000E54B797197F807B0B3F90A90B3F91A10F0
:10742000B3F908C0B3F91C8001FB09FA08FB1CA3DF
:1074300008FB09F801FB0C8143F3CF3340F6B83A5F
:1074400003FB0AF341F3CF3141F24C4C01FB0CF149
:1074500003EB010C5B421944CCF1000C4910DFF83E
:107460004C934FEA6C0C5B42CCF1000CC1F1000E66
:10747000A9F1060A40F2EE28BBF1070F80F0D08197
:10748000DFE80BF0FE0D559EE8FDFC00002AA8BFCA
:107490000221BBDA0028D4BF06210121B6E76146EC
:1074A00000F06EFA388DB98D05B20144B8780EB28D
:1074B00028B3BAF90000B028A4BF06F10C0006B248
:1074C0000ADA10F1B00FD1BFA6F10C0040F6B801F6
:1074D000484306EBE03006B2B9F90000B028A4BF7B
:1074E00005F10C0005B20ADA10F1B00FD1BFA5F119
:1074F0000C0040F6B801484305EBE03005B2002E21
:10750000B8BF002603DBB045B8BF40F2EE26002D21
:10751000B8BF002503DBA845B8BF40F2EE25A9B2ED
:10752000B0B200F0DDF90FFA80F800F07DB9114635
:10753000009800F025FA388DB98D06B2084405B2DE
:10754000B87828B3BAF90000B028A4BF06F10C003F
:1075500006B20ADA10F1B00FD1BFA6F10C0040F666
:10756000B801484306EBE03006B2B9F90000B02894
:10757000A4BF05F10C0005B20ADA10F1B00FD1BFBB
:10758000A5F10C0040F6B801484305EBE03005B228
:10759000002EB8BF002603DBB045B8BF40F2EE2690
:1075A000002DB8BF002503DBA845B8BF40F2EE258B
:1075B000B1B2A8B200F094F90FFA80F800F034B933
:1075C0000146704600F0DCF9388DB98D04B20144F3
:1075D000B8780DB230B3B9F90000B028A4BF05F1F6
:1075E0000C0005B20ADA10F1B00FD1BFA5F10C0002
:1075F00040F6B801484305EBE03005B26C48B0F9FD
:107600000000B028A4BF04F10C0004B20ADA10F1A3
:10761000B00FD1BFA4F10C0040F6B801484304EB11
:10762000E03004B2002DB8BF002503DBA845B8BF89
:1076300040F2EE25002CB8BF002403DBA045B8BF04
:1076400040F2EE24A1B2A8B200F04AF90FFA80F895
:1076500000F0EAB81946104600F092F9388DB98D5D
:1076600005B2084404B2B87850B3B9F90000B028A4
:10767000A4BF05F10C0005B20EDA02E080E036E0AE
:10768000CEE010F1B00FD1BFA5F10C0040F6B8016B
:10769000484305EBE03005B24548B0F90000B0289A
:1076A000A4BF04F10C0004B20ADA10F1B00FD1BF8C
:1076B000A4F10C0040F6B801484304EBE03004B2FA
:1076C000002DB8BF002503DBA845B8BF40F2EE256A
:1076D000002CB8BF002403DBA045B8BF40F2EE2465
:1076E000A9B2A0B200F0FCF80FFA80F89CE0714655
:1076F000604600F045F9388DB98D06B2084404B2F1
:10770000B87830B3BAF90000B028A4BF06F10C0075
:1077100006B20ADA10F1B00FD1BFA6F10C0040F6A4
:10772000B801484306EBE03006B22148B0F900004A
:10773000B028A4BF04F10C0004B20ADA10F1B00FB3
:10774000D1BFA4F10C0040F6B801484304EBE0308F
:1077500004B2002EB8BF002603DBB045B8BF40F22C
:10776000EE26002CB8BF002403DBA045B8BF40F2D2
:10777000EE24B1B2A0B200F0B3F80FFA80F853E0F3
:107780001846009900F0FCF8388DB98D04B2014418
:10779000B8780EB268B3BAF90000B028A4BF06F1F9
:1077A0000C0006B211DA05E0CC0000200601002032
:1077B0000C01002010F1B00FD1BFA6F10C0040F673
:1077C000B801484306EBE03006B23C48B0F900008F
:1077D000B028A4BF04F10C0004B20ADA10F1B00F13
:1077E000D1BFA4F10C0040F6B801484304EBE030EF
:1077F00004B2002EB8BF002603DBB045B8BF40F28C
:10780000EE26002CB8BF002403DBA045B8BF40F231
:10781000EE24A1B2B0B200F063F80FFA80F803E0F2
:107820000020F87040F2ED28DFF894902548DFF84A
:1078300098B099F8151069B3DFF890A0F979002392
:1078400001221AF83110FBF72BFFF87900230AEB1D
:10785000C000012201795846FBF722FF79791C48C4
:10786000002901880CBF21F4005141F4005101802E
:10787000184899F81530011D0A1D002B0CBF068011
:1078800004800D800CBF148016801348A0F800807F
:10789000BDE8F88FDFF844A0F979002301221AF837
:1078A0003110FBF7FDFEF87900230AEBC00001223E
:1078B00001795846FBF7F4FED0E700000C010020E8
:1078C0004C04002000240140002801404C0100200D
:1078D000202C0140342C0140402C01401401002098
:1078E0002DE9F001DFF894C0012500F148039CB2B6
:1078F00040F2EE228CF8035094429EBF40F2ED20FD
:10790000BDE8F0017047441AA4B2622C81BF1B3855
:1079100080B2BDE8F00170479FB200F13D031FFA4D
:1079200083F8002440F2DC56A1F11B0342450ED936
:10793000F01B80B2904205D98CF80340BDE8F001FD
:1079400098B270478CF80550BDE8F001704790423E
:10795000F2D301F1480087B297423EBF40F2D320F4
:10796000BDE8F001704780B23D3189B28A42E3D967
:10797000301A80B29042E5D9DEE70000CC0000204A
:10798000F0B4274E4FEA21420014C6E90A024FF034
:10799000000144BF02EB6000C6E90A10F06A00284B
:1079A00004DAB26A02EB6000C6E90A01D6E90A10FD
:1079B000084440F2EE27B842DCBFF0BC704740F20A
:1079C000EE2201FB02F3002808BF002122D0002193
:1079D0004FF0010C05460A4605E000BF4000521C6E
:1079E0004FEA4C0CD2B2984298BF212AF6D34208F3
:1079F00000244FEA5C0C95420CD8934224BF9B1A9A
:107A000061445208601C4FEA5C0CC4B2954298BFB6
:107A1000212CF2D3781AB162F062F0BC70470000FA
:107A2000CC0000202DE9F047524F90B03846FBF7CC
:107A3000B5FD514D2846FBF7B1FD01213846FBF756
:107A400098FD01212846FBF794FD6846FBF7A8FE48
:107A50004FF4803046114FF4602A4FF00109CDE910
:107A600002A600908DF8049000244FF004088DF8D1
:107A700005408DF8108069463846FBF7EDFD6846F5
:107A8000FBF78EFECDE902A68DF804908DF8054037
:107A90008DF8108069462846FBF7DEFD3846FBF777
:107AA0007AFE2846FBF777FEB9464846FBF7B5FD58
:107AB00007462846FBF7B1FD0742F6D10223012213
:107AC00000214F464846FBF718FE02231A460121C3
:107AD0003846FBF712FE0223032208213846FBF743
:107AE0000CFE0223042209213846FBF706FE02237E
:107AF000012204212846FBF700FE02231A46032137
:107B00002846FBF7FAFD0223032219462846FBF715
:107B1000F4FD0223042210212846FBF7EEFD01218B
:107B20003846FBF75DFD01212846FBF759FD012191
:107B30003846FBF728FD01212846FBF724FD0F4DB1
:107B40002846FCF7C1FA0B4806A94C3005900C48B2
:107B500081E811018020CDE909408000CDE90C6465
:107B60000B900E9405A928460F94FCF72DFB10B03E
:107B7000BDE8F087002401400028014008000240D1
:107B8000681100202DE9F04188B007A8FDF76BF8D7
:107B90004FF48050ADF81C0018208DF81F00474CA2
:107BA00003268DF81E6007A92046FCF7D3FFE114D9
:107BB000ADF81C1048208DF81F008DF81E6007A935
:107BC0002046FCF7C7FFDFF8F8804046FBF758FF78
:107BD000002501248DF816508DF817408DF81850A7
:107BE0000B208DF819408DF812508DF814008DF887
:107BF0001A508DF8135002278DF81B508DF8157010
:107C0000ADF8106004A94046FBF7C4FF4EF2E04611
:107C1000ADF8006041F60C00ADF80200701DADF843
:107C200004008DF80A5045F20C008DF80B408DF8D9
:107C30000C40ADF80600ADF808508DF80D406846D0
:107C4000FBF73AFFADF8006042F61C00ADF8020009
:107C50008DF80A40ADF8046042F20C008DF80B403C
:107C60008DF80C40ADF80600ADF808508DF80D40C9
:107C70006846FBF721FF43F20C008DF80A70ADF85F
:107C80000060ADF804608DF80B408DF80C40ADF845
:107C90000200ADF80600ADF808508DF80D406846BA
:107CA000FBF70AFF02214046FBF7A6FE0122022154
:107CB0004046FBF767FF08B0BDE8F08100080140CF
:107CC0000064004010B5002002F0C0F90121084610
:107CD00002F0C6F9012140F63D6002F0E5F901210C
:107CE000084802F0C9F901210420FCF789FF0121AD
:107CF0000548FCF785FF0121BDE81040C803FCF7EB
:107D00007FBF000007000002000230002DE9F04DA7
:107D10004FF0000846464546FCF742FDDFF800B448
:107D2000DFF800A40024ABF80040AAF80040FE48A9
:107D3000FE4F04803C80204602F0B8FC6420FCF733
:107D400061FAFB483C804480F94C00202070FBF72E
:107D5000E3FBF84F15E00220FCF726FA28B10220D9
:107D6000FCF79CF92078401C207002213846FBF774
:107D70005BFC30B102213846FBF7F8FB2078401C51
:107D8000207020780228E6D10120FCF73BFAEA496E
:107D9000E64B08681F88C0F34A123A441A8006EB83
:107DA000505086B260888988401CC1F34A1180B265
:107DB00029448DB260801028C6D3184640F69671CB
:107DC0000088DE4CA0F530502638884203D3E08985
:107DD00040F08000E081DA48DB4A4680D9480580DF
:107DE0000020014613689B0501D4491CC9B2401C00
:107DF000C0B2FF28F6D3642901D94FF0010884F8F6
:107E00000D80E08920F48060E081002002F04EFCCB
:107E1000C7490020CD4F48803888C007FCD038883B
:107E200020F00100388005E03A88D20702D0401CDB
:107E30004880F4E748880528F6D388460A4608892A
:107E400045F25001084390805189C04D41F05001E6
:107E50000835A8F8061028802E1D3180388820F0BB
:107E600001003880012002F021FC0AE03888000679
:107E700007D5002002F01AFCE08940F48060E08120
:107E800002E03888C007F1D0002002F00FFC3888EB
:107E90003B4620F0010038806420FCF7C1F91888C7
:107EA000000603D5E08940F48060E0816420FCF79F
:107EB000B7F9E08920F40070E08140054AD4002041
:107EC00002F0F4FB00204146A8F802003888C00701
:107ED000FCD0388820F00100388005E03A88D207CD
:107EE00002D0401C4880F4E748880528F6D308896A
:107EF00044F24002104388804A8942F04002A8F8C8
:107F0000062028803280388820F001003880012047
:107F100002F0CCFB0AE03888000607D5002002F00A
:107F2000C5FBE08940F40070E08102E03888C007BA
:107F3000F1D0002002F0BAFB388820F00100388030
:107F40006420FCF76DF93888000603D5E08940F419
:107F50000070E081002002F0A9FB00204146A8F853
:107F600002003888C007FCD0388820F00100388033
:107F700006E03A88D20703D0401CA8F80200F3E7D5
:107F800048881428F5D3E08910F4C06F6FD100221F
:107F90004FF490616E48FBF755FB4FF4E0416C489D
:107FA000FBF732FB4FF4E0416248FBF72DFB012168
:107FB0006748FBF71FFB01215E48FBF71BFB032112
:107FC0006348FBF792FB0323012206216048FBF77D
:107FD00067FB0323022207215D48FBF761FB0323B4
:107FE0001A4605215A48FBF75BFB388820F0010050
:107FF00038803888C007FCD0388820F001003880ED
:10800000B8F8080044F240010843A8F80400B8F8A2
:108010000A1041F04001A8F8061028803180388805
:1080200020F001003880012002F040FB0AE038888F
:10803000000607D5002002F039FBE08940F400700B
:10804000E08102E03888C007F1D04048018821F083
:10805000010101803E4F04213846FBF787FA0121D8
:108060003846FBF78EFB0020A8F802000CE03FE04A
:1080700036480088000607D5002002F017FBE0898B
:1080800040F40070E08105E004213846FBF7CCFAAB
:108090000028EDD014213846FBF7CDFABBF80020BC
:1080A00002EB1011ABF8001018213846FBF7C3FAA9
:1080B000BAF8002002EB1011AAF800101C21384673
:1080C000FBF7B9FA01461848028802EB111101804A
:1080D00004213846FBF74AFA01213846FBF751FBE9
:1080E000B8F80200401C80B2A8F802001028CBD3D8
:1080F000002002F0DBFAB8F8080046F260010843FD
:10810000A8F80400B8F80A1047F260031943A8F869
:10811000061028803180002002F0C8FA5D4619E080
:10812000EE000020F0000020F2000020EC00002013
:108130002C0000200028014068110020700300205E
:10814000C403002064040020080C0140102C0140EE
:1081500000240140BBF80020BAF800105746501A1E
:1081600000B2002800DA4042464E0FFA80FC308808
:10817000131A1BB2002B00DA5B420FFA83F80B1ABA
:108180001BB2002B00DA5B42DFF8FCB01BB245F2F9
:10819000757E4FF4804ABCF5A47F15DA4FF4A47CB9
:1081A000E04511DA63450FDA43F6B8639A420BD320
:1081B000994209D3984207D344F247139A4203D80D
:1081C000994201D8984218D9BBF80010714509D1DD
:1081D0002E48008828802E48008838802D48008846
:1081E000308017E0A5F800A0A7F800A0A6F800A02E
:1081F000E08940F08000E0810FE0BBF8004074456A
:1082000008D0224B1A80224A118022490880224934
:10821000012008702988514502D32888C0F5004103
:10822000484661F30F003988514501D3C1F500413B
:10823000328861F31F40524501D3C2F500424946DE
:1082400062F30F0183B2040C144AA34200D300145A
:108250001080B2F9003088B2984200DA1180B2F989
:1082600000004FF448414843001410800C494FF47B
:108270004D425043001408800A490880BDE8F04D83
:10828000FCF7D6B9F2000020920100208C010020FA
:108290008E01002090010020840100208801002030
:1082A000860100208A0100202DE9F8436846FCF78A
:1082B000DAFCFF20ADF80000DFF84C8100248DF8D7
:1082C000034069464046FCF745FC6846FCF7CBFC9A
:1082D00003254E4EADF800508DF8034069463046F8
:1082E000FCF738FCFF214046FCF782FC03213046B6
:1082F000FCF77EFC6846FCF7B6FC48278DF8037057
:108300004FF4E070ADF8000069463046FCF722FCFF
:108310006846FCF7A8FC4FF4E064ADF80040182074
:108320008DF803008DF8025069464046FCF712FCB8
:108330006501ADF8005069463046FCF70BFC21465C
:108340004046FCF755FC29463046FCF751FC684690
:10835000FCF789FCB414ADF8004004208DF803004C
:1083600069463046FCF7F6FB21463046FCF740FCF8
:108370006846FCF778FC4FF40870ADF800008DF803
:10838000037069463046FCF7E5FB6846FCF76BFC7A
:1083900010208DF8030001208DF8020040F61C40EB
:1083A000ADF8000069463046FCF7D4FBE400ADF8B8
:1083B000004069464046FCF7CDFBADF80050144D37
:1083C00069462846FCF7C6FB002261113046FCF7DF
:1083D00052FC002204213046FCF74DFC002208210B
:1083E0003046FCF748FC002210213046FCF743FCE5
:1083F000002221462846FCF73EFC0122D1023046ED
:10840000FCF739FCBDE8F88300080140000C01408E
:108410000010014038B54FF4A06001F06DFA18204B
:108420008DF8000000248DF801408DF802400125F0
:108430008DF80350684601F02DFA19208DF80000E0
:108440008DF801508DF802408DF80350684601F018
:1084500021FA12208DF800008DF801508DF80240AD
:108460008DF80350684601F015FA1E208DF80000C3
:1084700002208DF801008DF802408DF80350684607
:1084800001F008FA14208DF8000003208DF8010097
:108490008DF802408DF80350684601F0FBF906485C
:1084A00004800648018821F001010180018821F043
:1084B0008001018038BD000010080040102C0140F0
:1084C000F0B43D48018801F08F0101804FF4D27172
:1084D0000180394A40F2EE212C3211800024111F14
:1084E0000C80354D012314352B80111D0B802E1D62
:1084F00046F668013180371D47F668013980011D55
:108500004FF47C520A803A1D40F6880CA2F800C055
:10851000B2F800C04CF4805CA2F800C00A8822F0D7
:1085200070020A800A8842F020020A802A1F1188FD
:1085300021F080011180DFF880C040F277110CF14A
:10854000340CACF800100CF1040CACF800100CF179
:10855000040CACF800100CF1040C40F2ED21ACF866
:108560000010154945F60C4C4431A1F800C0B1F893
:1085700000C04CF4807CA1F800C0B0F800C04CF002
:10858000010CA0F800C0368848F68F7006400B48F2
:1085900006813E8826F070064681088840F4004037
:1085A00008808120111F08802B8010881480F0BC67
:1085B000002002F07BB80000002C01402C000020BD
:1085C0003EB54FF6FF70ADF8040045F6BF50ADF86C
:1085D00000004FF40070ADF806000020054CADF827
:1085E00002006946204602F00FF90121204602F000
:1085F000E9F83EBD000400403048016941F0040143
:108600000161016921F0040101612D4A40151080CA
:108610002B494FF6FF702C31088029482030018803
:1086200021F001010180264918310B8823F0F30362
:108630000B800B8843F0F1030B80038823F00A03BF
:108640000380038843F0030303800B8823F00C03AB
:108650000B80038823F0010303800B8843F003039E
:108660000B80018841F0010101801549002028316B
:10867000088013490120143108801148083001880E
:1086800021F007010180011F0B8843F080030B805C
:10869000018821F070010180018841F040010180D2
:1086A000018821F007010180018841F00401018067
:1086B000108840F004001080704700000010024055
:1086C000000800404FF0E020016941F00401016121
:1086D00009494FF47A720968B1FBF2F14161074A26
:1086E000F02182F8141D016941F001010161016965
:1086F00041F0020101617047000000200FE000E03E
:1087000070B5234D4FF49064002221462846FAF7B5
:1087100099FF00212846FAF76DFF04212846FAF751
:1087200025FF01212846FAF7E0FF1A4E01213046C5
:10873000FAF7DBFFA9142846FAF766FF00230122A7
:1087400006212846FAF7ACFF002301220721304614
:10875000FAF7A6FF01212846FAF74CFF012130461F
:10876000FAF748FF04212846FAF700FF01222146C4
:108770002846FAF767FF084C0121204602F01CF852
:108780002046BDE870400122114602F033B80000D7
:108790000024014000280140002C014010B5FFF7E3
:1087A0008FFEFFF73FF9FFF727FFFFF709FFFFF7FE
:1087B000ADFAFFF7A5FFFDF7F5FEFFF72BFEFFF77C
:1087C000E1F9FFF77FFFFAF7A7FEBDE81040FCF7DD
:1087D0006DBC0000F0B5314A314BD078810614D51C
:1087E000C00612D45889042802D2401C58810CE0DB
:1087F000D08940F40060D081FEF73CFD294901207A
:10880000C870D07840F01000D070908B0A2802D841
:10881000401C908303E02448FF21A0F8C210234DA0
:10882000234E244C2F782448002107B3D77827F013
:108830000107D7704170B68A322E02D92678012EF0
:1088400000D029705978837899420BD12178032977
:1088500008D09178C07801F00101814202D1D0782E
:10886000C00603D5D07820F00100D070F0BDB58AE5
:10887000642D0ED21D78AD0709D5D57845F00105D8
:10888000D5705D788570957805F00105C5704170EB
:10889000D8E7D17821F00101D170D3E7700300202F
:1088A00090040020280000208C02002022000020DC
:1088B0001C04002065020020C40000202DE9F05FA8
:1088C000DFF808B4BBF80010BBF80C00814234BFDD
:1088D0004FF0010A4FF0000ADFF8F483FD4800264C
:1088E000A0F11E04B8F80030227820F81230521C93
:1088F000D2B22270042A08BF2670B0F90020B0F965
:1089000002301A44B0F90430B0F90600184410449B
:108910008010A0826078F04FF04D4FF003090128DD
:1089200014D02E736078022818BFA68000F0C6828B
:10893000607803281CBF6078042800F04983E88928
:1089400010F4807F00F0138300F019BBBBF80A001D
:10895000884228BF268211D2208A10283CBF401CA2
:1089600020820BD301208BF81E00E88940F0200004
:10897000E881002001F09AFE84F80190D84801783F
:10898000012920D0B8F90220B4F914108A4259DA2A
:10899000881A00122E730128B8BF012002DB0428B8
:1089A000C8BF042082B2B4F904108A42A8BFA680CE
:1089B00080F2FF81081A00B2A0800028C4BF401EC8
:1089C000A08000F0F6B906702E73BAF1000F1CBF3C
:1089D000B4F904001028C4BF1038A080687B0028B8
:1089E0001CBFB8F900000D2880F2E381002001F0DF
:1089F0005DFE6078032818BF6670687B18B1E8894F
:108A000040F48070E881B748007828B1E88940F0E8
:108A10000400E88184F801909BF81D0028B1E889E2
:108A200040F04000E88184F801909BF81E00002887
:108A300000F0BF81E88940F02000E88184F80190CF
:108A400000F0B7B9E88950B9A6480078002801BFFE
:108A50009BF81E0000289BF81D00002856D02E739E
:108A6000BAF1000F12D0B8F9001048110428C8BF9D
:108A7000042002DC002808BF0120052937DDB4F9F5
:108A800004108142D2BFA680081AA080B8F9000065
:108A90000D2802DAB88A962804D9B4F904000A2805
:108AA00080F28781002001F001FE6078032818BF62
:108AB0006670687B18B1E88940F48070E881894865
:108AC000007828B1E88940F00400E88184F801903A
:108AD0009BF81D0028B1E88940F04000E88184F847
:108AE00001909BF81E00002800F06381A2E7A18995
:108AF000491C89B2A1811029CCD3B4F90410814258
:108B0000C6BF081AA080A680A681C3E77648007871
:108B1000E8B12E73BAF1000F1CBFB4F904000328AA
:108B2000C4BF401EA080B8F900001A28A4BFB4F941
:108B300004000A2880F23D81002001F0B7FDE88999
:108B400040F00800E88184F8019000F032B9B4F9EF
:108B50000230B4F90400984203DA0A2B08DD00F071
:108B60002AB90A2BC4BF03F16401814200F3FA80E1
:108B7000BAF1000F7ED0B98A46297CD3B7F9161016
:108B80003A8C914277DB6A7812F0040F1CBF2A7985
:108B9000002A05D16A7B002A04BFEA7F002A0BD095
:108BA000524B4FF4007C4FF00102A3F800C04FF08D
:108BB000400CA3F804C012E07B8C4FF000029942F5
:108BC000ACBF4FF4807C4FF0800C484BA3F800C042
:108BD000ACBF4FF0200C4FF0100CA3F804C095F878
:108BE0000CC0434BBCF1000F18D14FF00A0CA4F895
:108BF00018C04FEAA11CCCF10009A4F81A90B3F9EF
:108C000000C0E14500F3FE81E0824FF0010C85F8E1
:108C10000CC04FEAC03C3548C0F814C0208B002A75
:108C200014BF00EBE10000EB2110C0F1000001B225
:108C300018BF6183B4F91A008842B8BF401CC8BF8E
:108C4000401E00D06083294AB4F91A10B3F900001D
:108C500000F010FFA080B4F9161040F2DC528142FF
:108C6000C8BF668204DC638A93429CBF5B1C63823C
:108C7000CB1C01E05DE03DE0984202DA638A93425A
:108C800006D3208B642838BF401C52D2208350E08A
:108C9000821D8A4206DC218B00291CBF491E2183CC
:108CA000E08246E07A890F2A43D9E289521C92B2C7
:108CB000E281202A3DD3E68181423ADDE082208BA9
:108CC000002818BF401E34D0E0E7000064040020F4
:108CD00084040020820200201C0400207003002075
:108CE000D2000020A6010020A4010020E004002002
:108CF000EA0000202E736189491C89B2618107292D
:108D000017D96681B8F900100D2903DD0D39091155
:108D1000012901DA012102E00429C8BF04218842A7
:108D2000A6BF401AA080A680B4F904009842C0F201
:108D30006C81B4F902000A283BDCB88A462804D9C1
:108D4000B7F91600398C884233DCB8F900000D28D9
:108D5000A4BFB4F904000A282BDC002001F0A6FC13
:108D6000667026E02E736189491C89B261810F29E2
:108D70001FD9BAF1000F18BF98421ADD6681B8F901
:108D80000010052915DD0D2903DD0D390911012913
:108D900001DA012102E00429C8BF0421C21A8A4273
:108DA000A6BF401AA080A380B4F904009842C0F284
:108DB0002E8126810CE1DFF85CC22E73BCF814C052
:108DC000BCF1780F98BF4FF0080C0FD9DFF844C200
:108DD000924FBCF80A90DFF840C2B9F10A0F9CF834
:108DE00001C017F80CC088BF4FEA5C0C6681DFF841
:108DF0003092278929F81710791C89B221816145A1
:108E00005BD30021ACF10109B9F1000F16DD854FEC
:108E10001CF0010F08BF37F9021FB7F902B04FF07D
:108E2000000A5FEA690908D037F904EF5944B7F935
:108E300002B0F244B9F10109F6D15144BCF1010785
:108E400004D4DFF8DC9139F917703944083191FB0B
:108E5000FCF1511A41F3CF1126810129B8BF01213C
:108E600004DB2A898A42B8BFB5F90810694AB2F909
:108E700016C0178BBC45A8BF002118DAD28CBA1ACD
:108E8000624514DAA7EB0C02521CC2F34F028A426D
:108E9000B8BF11B2B8F90020B4F81CC0A2EB0C0C9A
:108EA0000FFA8CFCBCF11E0FC8BF0021A2831A1A56
:108EB0009142B4BF0844401CA08089E05A4AB7F9E7
:108EC000160012680028B8BF4042504301F072FEFD
:108ED00080B244F6E7418842C8BFA18005DCB0F506
:108EE000C87FB8BF4FF4C870A080B5F906000A2843
:108EF0003BDDE989C1BBB4F90410884235DB4B4B3B
:108F000001F5FA60B3F930208242C8BF02461A86E2
:108F1000474AB2F930308342C8BF108606DC454B61
:108F2000B3F910208242C8BF02461A824248DFF8D5
:108F30000C8146614248C8F814600680FDF754F879
:108F4000F88A002808BFFDF741F8B4F904003D494C
:108F50000880C003C8F8140000F01CFC01206070F9
:108F6000A87701F0A3FBE3E4FFE76670E0E4617833
:108F700004291FBF697B002940F48070E88180B21A
:108F800010F0040F06D13049097800291CBF40F0C9
:108F90000400E88180B210F0400F06D19BF81D104C
:108FA00000291CBF40F04000E88180B210F0200F83
:108FB00006D19BF81E1000291CBF40F02000E8815C
:108FC0000004000C04D084F80190002001F06EFB36
:108FD000E88910F4885F06D0697B21B930F48850A5
:108FE000E88108BF6670B4F904000028BCBFA68001
:108FF000BDE8F09F44F698118142B8BFA180BDE85A
:10900000F09F00BFA4F81AC0FEE5A38091E6A380FC
:10901000CFE600001C04002090040020FCCB0008D8
:10902000541200205212002004020020C403002029
:1090300090030020F6030020F8040020E004002044
:10904000E6000020E8000020A60100202DE9F04104
:109050001E4C20781E4B1F4A01280AD0D8891E4D6D
:1090600010814FF00006E88910F0600F03D0D67031
:1090700029E0188AF3E71988B2F808C0012761458A
:109080000CD29670D1780F2903D2491CD170BDE85B
:10909000F0815F7740F04000E881F8E7D670B3F8E0
:1090A0000AC061450FD99178022902D2491C9170FA
:1090B000EDE79F7740F02000E881002001F0F6FA0C
:1090C00003202070E3E79670E1E7000065020020CE
:1090D00064040020780000207003002010B5FDF724
:1090E00023FAFBF7CDFDFCF713F8FFF7E7FB00F0E1
:1090F000F3FFFEF757F9FCF73FF9BDE81040FBF727
:109100001DBEFCF75BBA000006498968C9094143E6
:109110000A20B1FBF0F004490988B0FBF1F080B2FD
:10912000704700004C0400201C0400202DE9F04191
:10913000294C208B1E2801D800200CE0322801D8B1
:10914000052008E0642801D80A2004E0962801D808
:109150000F2000E01420E0840A20FFF7D5FFE08311
:109160001E48408EFFF7D0FFA084E08B4FF6FF71C2
:10917000C0EBC000208401EA4000608418483C2114
:109180001A4F007DB1FBF0F0A08516481649027811
:10919000C87862F3C300C870A48AB4B1B868401C30
:1091A000B860012811D002F055FC05460E46F8685B
:1091B00002F050FC0E4A0F4B02F060FC2A46334688
:1091C00002F07CFA02F002FCF882388BA04200D256
:1091D0003C83BDE8F08100001C0400208C020020CC
:1091E0004C04002022000020700300209C0400207A
:1091F000CDCCCCCCCCCC0C402DE9F0473D4F6421FC
:109200003888484302F026FC3B4A3C4B02F056FAB1
:1092100002F0DCFB3A4C86B2BE80B4F900000025B7
:10922000DFF8E080DFF8E090002816DD00EB80003A
:10923000400002F00FFC354A354B02F03FFA02F0D5
:10924000C5FB80B26081282808D998F8000005285D
:109250001AD2401C88F8000002E0658188F80050AE
:1092600060892C4D46434FF47A7096FBF0F0F880FD
:109270002878294C80064FF4806108D501222046C9
:10928000FBF7F9FC012207E089F81F50E8E700220C
:109290002046FBF7F0FC002208212046FBF7EBFC00
:1092A00099F80D00B8B11C4D08352868400701D564
:1092B000002200E0012204212046FBF7DCFC2868A4
:1092C000C00601D5002200E001222046BDE8F0479B
:1092D0001021FBF7D0BC2878800605D50122042197
:1092E0002046FBF7C8FCEFE7002204212046FBF7ED
:1092F000C2FCE7E76404002027A74D843CE07E40E1
:1093000084040020C400002070030020888E556370
:109310006DE35D4090040020000C01402DE9F84F02
:10932000FA48FB4B0A210688B0F802A0188EFA4AC8
:10933000B0FBF1F0F7494883202182F82310F74A67
:10934000C0B2894682F82200202802D9104680F84F
:109350002210EF48F24C1221B0F8B20048B9EC48A4
:10936000B0F8B6202AB190F8B10010B120721228DE
:1093700000D92172EB480078642520B96E2E02D8FE
:10938000E948007820B1207A00EB800080000AE1F3
:10939000E648C078C0076FD1E5484778781E0928AD
:1093A0006AD2DD48DFF870B3C0790BF1240BE8B363
:1093B000D94A44F698131146012891F82D1001FB63
:1093C00003F85AD0022874D0207A6421484302F06E
:1093D00041FBD84AD84B02F051FB0022D74B02F098
:1093E0006DF902F0F3FACC498881B8FBF5F0A1F8E9
:1093F0000890C885DFF82483414601F1190098F8E8
:10940000002023310091002A75D0434603F10F015B
:1094100093F82C3044F6981C03FB0CFB012A68D00F
:10942000022A67D0207A6421484300E01CE002F061
:1094300011FBC04AC04B02F021FB0022BF4B02F0DF
:109440003DF902F0C3FAA8F8060098F82200A8F83F
:109450000200BBFBF5F0A8F82E00B4480079002804
:109460007DD0B8F80600ABE0AB48DFF8AC821A302C
:10947000395CA8F8081020E091E0A749A2F808900C
:109480001031207A795C9346484302F0E3FAA94A06
:10949000A94B02F0F3FA0022A84B02F00FF902F0F8
:1094A00095FAB8FBF5F1ABF80C00ABF82E10A1E77C
:1094B000FFE7DFF86482A8F80890207A6421484327
:1094C00002F0C8FA9B4A9C4B02F0D8FA00229B4B50
:1094D00002F0F4F802F07AFAA8F80C0017F80B0082
:1094E00044F698114843B0FBF5F1A8F82E1081E737
:1094F00001E01EE034E0395CA8F80210207A642113
:10950000484302F0A7FA8B4A8B4B02F0B7FA0022CD
:109510008A4B02F0D3F802F059FAA8F80600009836
:1095200044F69811385C4843B0FBF5F1A8F82E10CA
:1095300093E798F82220A8F80220207A795C484323
:1095400002F088FA7B4A7C4B02F098FA00227B4BAF
:1095500002F0B4F802F03AFAA8F8060079E71BE046
:109560003A5CA8F80220207A795C484302F072FA4B
:10957000704A714B02F082FA0022704B02F09EF8A2
:1095800002F024FAA8F80600009844F69811385C16
:109590004843B0FBF5F05EE75F48808910E0207A31
:1095A00000EB8000400002F055FA624A624B02F084
:1095B00065FA0022614B02F081F802F007FA80B2EE
:1095C00055490A89202A01D9A1F8089053494A88A7
:1095D00091F822108A4201D9504A5180584909789D
:1095E000584FDFF864C10129BA8808D1BCF80A10C5
:1095F00029B18A4206D21E2904D91E3911E0ACF8DD
:109600000A2010E08A4203D20A2901D90A3908E067
:109610008A4203D2052901D9491F02E08A4202D2B7
:10962000491EACF80A103A49B1F8C21064290ED8A4
:109630000A2920D2022912D3A0F1EF02891E514338
:10964000CA1701EB5271EF2202EBE10111E0BB8A74
:10965000BCF80A108B420ED9FA8A8A4201D9EF214E
:109660000AE09B1A8A1AA0F1EF014A4392FBF3F138
:10967000EF3109B200E001B2244A64236E2E17884C
:109680005288A7F15F08A2F16E0B08FB03F70BFBF2
:1096900003F902D8BAF1820F01D9EF2018E05F2E4A
:1096A00002D8BAF16E0F12D90FFA88F30FFA8BF2C3
:1096B000934203DB0F2297FBF2F202E0142399FBA3
:1096C000F3F2A0F1EF035A43B2FBF5F2801A00B2B5
:1096D000814200DC0846A080207A02F0BBF91B4AD8
:1096E0001B4B02F0CBF900221A4B02F0C7F94FF0E6
:1096F000FF3202F08CFD02F039F900B26E2E02D872
:10970000BAF1820F28D9002038E000001A000020AA
:109710008C0200201C040020C403002090030020C1
:1097200084040020A5010020A40100207003002073
:1097300090040020888E55636DE35D400000594021
:10974000650200206404002090000020581678650F
:109750008157564000001C405F2E02D8BAF16E0FB0
:109760000CD9D84503DB0F2197FBF1F102E014215E
:1097700099FBF1F14143B1FBF5F1401AE080034858
:109780000349C08DC881BDE8F88F00009003002018
:10979000F60300202DE9F041314A324F324CD08D92
:1097A0003880E07B08B106202081B2F8B2002F4D4E
:1097B0004FF6FF7610B9B2F8B60090B120896FF07D
:1097C000040100EB800001EB400080B2FFF79CFC3D
:1097D0006081688800EB800006EA4000FFF794FC97
:1097E00013E012F8BB0F00EB4001C1EBC01006EA1A
:1097F000C00000F043F86081107800EB4001C1EB3D
:10980000C01006EAC00000F039F8A8801848194ACC
:109810000188388B1268504301F0CCF900EB40000E
:1098200040016421B0FBF1F0134AD178C90701D09F
:109830003C2108E0117909B1698800E0218901EB38
:10984000810106EA4101B98344F69811884203D8A0
:109850004FF44871884200D208465081BDE8F0813B
:109860008C0200201C040020C40300209003002070
:109870006404002004020020700300200349C9682A
:1098800041433C20B1FBF0F080B270474C04002013
:10989000FEE7704730B50F23C27801780125F2B199
:1098A000144A126801F1E02102F4E062C2F5E062BC
:1098B000120AC2F10404D3404278A24084781C40CA
:1098C0001443220181F80024007800F01F018D402C
:1098D0004009800000F1E020C0F8005130BD01F0E7
:1098E0001F0085404809800000F1E020C0F8805149
:1098F00030BD00000CED00E0024908430249086059
:10990000704700000000FA050CED00E0024A11402B
:10991000014302480160704780FFFF1F08ED00E02F
:1099200070B5144A09200021108013480469436867
:1099300023441D0C55809380036823441C0CD48061
:10994000138183681C0C54819381008BD08100208B
:1099500032F81030401C194480B289B21328F7D372
:10996000D18414220349054800F066FC0449002014
:10997000887070BD181000209C04002000E80008CA
:109980002800002070B53448344C818A207B23297C
:1099900001D9012801D8C82112E03C2901D90228A7
:1099A00001D8B4210CE05A2901D9032801D8A021FB
:1099B00006E0782901D9042801D88C2100E078211B
:1099C000274A1268274D02F020024FF6FF762A80C0
:1099D000AB88B34201D25B1CAB8000235AB96E88BE
:1099E0004EB1AE886681AB80FF2804D2401CC0B265
:1099F0002073012812D06689A888864200D8608129
:109A00006A8060890122884203D21749B1F8501058
:109A100031B12381237384F8322070BD5020EEE7EA
:109A2000022801D2114802E01149B1FBF0F0642193
:109A3000B0FBF1F00004000C208100D12281207BDA
:109A4000617B401C884201D384F832302089C828C9
:109A5000E3D9C820208170BD1C04002090030020A1
:109A6000080C0140620000208C02002085450100A6
:109A70000A8B020030B4081AB2F90010136901FB16
:109A800000FCB2F9041048435169C417081844EBAC
:109A9000E1714FEAE3741D1A8C4106DBD368DC17D1
:109AA000C51AA141A8BF506101DA1846536160444C
:109AB000B2F90A10C0138142AABFB2F908100846D1
:109AC0008142C8BFB2F9080000B230BC7047000044
:109AD0001A490020C989CA0701D18A0701D5032084
:109AE00028E04A0701D5042024E0CA0601D5432016
:109AF00020E08A0601D5D0201CE00A0603D48A059E
:109B000001D44A0501D5412014E0090501D5802082
:109B100010E00B490988B1F5BA6F01D8112009E0AE
:109B200008490A886E2A01D3A12003E049888229C6
:109B300000D3A6200449087270470000700300207B
:109B4000F60300201A000020900400202DE9F043C5
:109B5000474A05204FF01208507046480122474BF3
:109B600000F80D2F444A4FF0C809142482F80880E9
:109B700002229A70424B01223C255A82FA229A8292
:109B8000A3F816904FF4C8721A834FF496725A8352
:109B900040F28A229A834FF4C872DA8352001A8400
:109BA0004FF4FA725A8440F2B6329A840A238370D0
:109BB000C4701E2202712822427132228271C57144
:109BC00046260672502747724FF05A0C80F80AC09A
:109BD0006422C2728375C5754125057646764B258C
:109BE0008576C7765525057780F81DC05F25857772
:109BF000C2770C22027342730D22002182730F225E
:109C0000C2731122027480F8118084741622C27407
:109C10001722027519221B4C42750325A5701A4C98
:109C200000F80D5D194E628342187418D77B2774B3
:109C300092F8237084F82470491C527EC9B2A2762F
:109C40000A29F1D31248F5710621A0F81290017586
:109C5000437040F2DC5101824FF42071C1800D4904
:109C6000002008800C4908808870C870BDE8F08327
:109C7000700300209003002084040020640400206E
:109C8000F6030020900400201C040020C4030020E0
:109C90004C040020140000201600002070B54E4D2A
:109CA0004E490024A8784870A888122802D90020BC
:109CB0004B4901E001F0CEFE01F088FE49490872EF
:109CC0004949A8798870494805EB440100EB4402F2
:109CD000641CB1F86410E4B251820A2CF4D3444AF3
:109CE000002005EB40011318401C91F8C810C0B2C9
:109CF000D9730A28F5D3002005EB40011318401C46
:109D000091F8DC10C0B259760A28F5D3002005EB93
:109D10004001B1F8F010642900D964211318401CE7
:109D2000C0B283F823100A28F1D3324995F8040110
:109D3000887095F80601507395F8080110702E4A46
:109D4000002005EB40011318401C91F82C11C0B203
:109D500019740A28F5D3002005EB40011318401CA4
:109D600091F84011C0B299760A28F5D3002005EB8E
:109D70004001B1F85411642900D964211318401C22
:109D8000C0B283F824100A28F1D395F868011B4962
:109D9000D071B5F86A0148831948B5F8901141822D
:109DA00095F89211017595F894114170B5F89611D6
:109DB0000182B5F89811C1801249B5F89A0108805E
:109DC0001148B5F89C11018095F89E11817095F8A5
:109DD000A011C17070BD0000D809002070030020E0
:109DE000000032408404002064040020F6030020B8
:109DF0009003002090040020C40300201C040020D5
:109E00004C040020140000201600002070B5534AB6
:109E100000210C2010805248544B4078508051480B
:109E2000007A908050488078D080084603EB400448
:109E300002EB4005401C648A80B2A5F864400A2801
:109E4000F4D34B4B00201C1802EB4005401CE47B74
:109E500080B2A5F8C8400A28F5D300201C1802EBF0
:109E60004005401C647E80B2A5F8DC400A28F5D38A
:109E700000201C1802EB4005401C94F8234080B2DF
:109E8000A5F8F0400A28F4D33A488078A2F80401F3
:109E9000587BA2F806011878A2F80801364B00207A
:109EA0001C1802EB4005401C247C80B2A5F82C4114
:109EB0000A28F5D300201C1802EB4005401CA47EA4
:109EC00080B2A5F840410A28F5D300201C1802EB07
:109ED0004005401C94F8244080B2A5F854410A285B
:109EE000F4D3D879A2F868012448408BA2F86A011B
:109EF0002348438AA2F89031037DA2F89231437837
:109F0000A2F89431038AA2F89631C088A2F8980189
:109F10001C480088A2F89A011B480388A2F89C31CB
:109F20008378A2F89E31C078A2F8A00100204FF4F7
:109F3000C77332F81040401C214480B289B2984265
:109F4000F7D9A2F81E134FF4C87204490F4800F065
:109F500073F90F490020087070BD0000D809002077
:109F6000700300208404002064040020F603002015
:109F70009003002090040020C40300201C04002053
:109F80004C040020140000201600002000E000080F
:109F900028000020254810B5B0F8C4402448254AC0
:109FA0000023B0F90000B2F9301054B9148944B15B
:109FB000947B34B192F832401CB91F4CE478E4062B
:109FC0000AD5814200DD1086B2F93000802801DD1B
:109FD000803828E0138610BD184C8142237000DAC7
:109FE000108617498B8A502B02D9B0F5FA6F04DA24
:109FF000144880788000001D07E04889202801D996
:10A00000202002E0082800D20820B2F930304FF4B6
:10A01000C8718B4200DA1186B2F930100844D18D34
:10A02000884200DB88B2108610BD00008C02002040
:10A03000680200209003002070030020220000200E
:10A040001C0400209004002070470000034A51685F
:10A0500021F440410143516070470000001002406C
:10A06000044A0029516901D0014300E08143516154
:10A070007047000000100240044A0029D16901D055
:10A08000014300E08143D1617047000000100240AD
:10A09000044A0029116901D0014300E081431161A4
:10A0A0007047000000100240044A0029916901D065
:10A0B000014300E0814391617047000000100240BD
:10A0C000044A0029D16801D0014300E08143D160F6
:10A0D000704700000010024070B5FBF7BFF9494A15
:10A0E00049484FF0010CB2F91A10B0F9000001FB19
:10A0F00001F4002812DD884226DD4043031B0020C6
:10A1000010214D1E0CFA05F10E18B1B249439942C7
:10A1100098BFB0B215F0FF01F3D115E018BF884227
:10A1200012DA4043031B00211020401E0CFA00F5F8
:10A130000D44AEB276439E4298BFA9B210F0FF0024
:10A14000F3D14842908300E090833048304B4FF089
:10A150000005C07810F0010F2BD1B2F91C0000FBF4
:10A1600000411C78012C24D1182922DDB1F1805F37
:10A170001FD228490978E1B9274909880C2903D851
:10A18000264909880C2914D99178A1B1B0F5804FDE
:10A19000C8BF40F2651006DC40F2651148438013E9
:10A1A0001128B8BF1120B2F91E10814219DA1079B6
:10A1B000B8B1957015E0B0F5804FC8BF40F27D3062
:10A1C00006DC40F27D31484380132C28B8BF2C2098
:10A1D000B2F91E10814204DD1079002818BF82F800
:10A1E00002C01878042828BF70BDDFE800F002091B
:10A1F0000202002000F05AFABDE87040FBF74AB9AD
:10A2000070BD0000CC000020680200207003002018
:10A210006502002099010020BA010020BC01002045
:10A2200010B5002305E030F8024B21F813405B1C09
:10A230009BB29342F7D310BD2DE9F05FA0F100640B
:10A24000154688468246B4F5803F50D2FAF746FB61
:10A25000A70AC4F34806C6F50074A54200D82C46E8
:10A26000DFF890B04FF0006000EB872081464FF49C
:10A2700000722049FFF7D4FF00204FF6FF7206E07E
:10A2800033183BF81310914203D1401C80B2A04216
:10A29000F6D3A04223D24846FAF7C4FA00205A4621
:10A2A00006E038F810108319401C22F8131080B211
:10A2B000A042F6D348464FF400720E4900F01CF855
:10A2C000A54210D0281B08EB4408A244002685B202
:10A2D0004FF400747F1CA542C4D82C46C2E7224626
:10A2E00041465046EAE7BDE8F05FFAF7D1BABDE86B
:10A2F000F09F0000D80500202DE9F04116460F46DA
:10A300000546FAF7EBFA2846FAF78CFA04280BD13F
:10A31000002407E037F814102846FAF7C1FA641C45
:10A32000A4B2AD1CB442F5D3BDE8F041FAF7B0BA1F
:10A33000704700001D48016841F4803101600168E8
:10A340008903FCD51A490A6842F010020A600A68BB
:10A3500022F003020A600A6842F003020A604168C0
:10A360004160416841F440514160416841F4C0613D
:10A370004160416821F47C114160416841F424113D
:10A380004160016841F08071016001688901FCD57C
:10A39000416821F003014160416841F002014160E0
:10A3A0004168C1F381010229FAD1704700100240CF
:10A3B000002002402DE9F0413D4E3E4FF08A10B1A1
:10A3C00042F2107004E0387D01281DD04FF47A70FD
:10A3D00039493A4DDFF8E880CA88E98800244FF609
:10A3E000FF73B2F5E16F1DD2AA88824201D2521CDE
:10A3F000AA8092B2012A0AD0824203D3EC602C6177
:10A400007380F3802C811DE040F6B830E0E7814294
:10A4100002D20120287003E00021404600F0F2F94A
:10A42000EC80EFE72A890A2A02D2521C2A8100E036
:10A43000AC80814202D2491CE98003E0EC602C61CF
:10A440007380F3802878002830D0B08A32284046C4
:10A4500008D800F0C6F9C5E90304397D414371808D
:10A460006C7013E000F0BDF92969401AE8600844F7
:10A4700028616878401CC0B26870397D884209D371
:10A480006C7040462C6100F0ACF9708000214046B1
:10A4900000F0B8F9387DA9894843F080387820B1B8
:10A4A000B878052801D2401CB8702C70BDE8F08146
:10A4B0001C0400204C0400201A0000209000002002
:10A4C000000400402DE9F00FDFF848A1524EBAF920
:10A4D0000020B6F906709742B8BF3A467FDB4F4B73
:10A4E000DD8B4F4B00EBC50C8C45B3F900300DD81C
:10A4F0009A427BDC0A282ABF081A8020042888BFD9
:10A500000420824288BF101A24D867E0434CDFF849
:10A5100014C105EB010BB4F81C90BCF90040DFF846
:10A5200008C14FF00008834516D29A4269DB00BF8C
:10A53000B6F90A009042C8BF024650DCBCF80000E1
:10A54000484400B2ACF80000A042A8BFACF80080BC
:10A5500045DB501C02B242E081420ED29A4252DBED
:10A56000BCF8020000EB990000B2ACF80200A04277
:10A57000A8BFACF80280ECDA31E030D900EB8509F5
:10A580004FF4FA74894538BF0A2410D300EB45090B
:10A59000894538BF32240AD305EB0009894538BF05
:10A5A000642404D300EB5500884238BFC824F07FF0
:10A5B000002806BFF07810F0010F32249A4224DC04
:10A5C000BCF80400401C00B2ACF80400844206DC75
:10A5D000ACF80480002AC8BF501EBBDC0022BA427F
:10A5E00015DC00BF44F69810824200E007E0C8BFC7
:10A5F00044F69812AAF80020BDE8F00F70471A46FA
:10A6000078E71A4694E71A46AAE71A46D8E73A4680
:10A61000E8E7000066020020700300201C04002010
:10A6200068020020EA0000204C00002001490120BF
:10A63000087070475E0300200C48016841F001017A
:10A64000016041680A4A114041600168094A1140AD
:10A650000160016821F480210160416821F4FE015C
:10A6600041604FF41F018160FFF764BE001002409B
:10A670000000FFF8FFFFF6FE10B58021084800F04B
:10A680009EF8002000F012F8FAF704FF0548C1898F
:10A6900041F01001C18104490320087010BD000081
:10A6A000002C01407003002065020020054A11883B
:10A6B0004FF6AA23194010B140F2555001431180C2
:10A6C00070470000202C014010B501210D4800F01A
:10A6D00073F8FEF703FD0220F9F766FD00280FD09E
:10A6E00002210948F8F7A0FF002809D002210748F5
:10A6F000F8F79AFF002803D0BDE81040F8F70CBF28
:10A7000010BD0000002C0140002401400028014041
:10A7100010B510218C06204600F065F898B1102184
:10A72000204600F04CF8204600F058F8094A5188BD
:10A73000884201D9411A03E04FF6FF73591A0144C8
:10A740001180508010BD2046BDE81040012100F06E
:10A7500033B800006800002070B5144D0121284670
:10A7600000F041F860B10121284600F025F81048BA
:10A77000818C2D2928BF70BD818C491C818470BDBE
:10A780000221284600F018F80A4C208820F0020028
:10A790002080FBF731FC208840F002002080284612
:10A7A000BDE87040022100F007B80000000800403A
:10A7B000940100200C080040C94301827047C9433E
:10A7C000018270470029018802D041F0010101E0B7
:10A7D00021F0010101807047808E7047B0F8400081
:10A7E0007047808C704702460020128A0A4200D0CF
:10A7F00001207047002A828901D00A4300E08A4381
:10A80000828170478184704730B502881B4C1C4D93
:10A81000A0420DD0A8420BD0B0F1804F08D0194B08
:10A82000984205D0184B984202D0184B984203D159
:10A8300022F070034A881A43154B984206D0154BF4
:10A84000984203D022F44073CA881A4302808A884F
:10A8500082850A880285A0420AD0A84208D00E4A02
:10A86000904205D00D4A904202D00D4A904201D14B
:10A87000097A01860121818230BD0000002C01404F
:10A88000003401400004004000080040000C00407B
:10A89000001000400014004000400140004401400E
:10A8A0000048014070B5414D2878002876D000243A
:10A8B0002C70E878401CC0B2E870012812D1EC700E
:10A8C000FCF750FCFFF75EF8FFF774FDF9F768FA44
:10A8D000FAF7E2FAFBF7A6FA00F0EAFCF9F7ACFCAB
:10A8E00000F042FA6879401CC0B26871052806D1B0
:10A8F0006C7100F099F8F9F799FA00F0C5FDA879A4
:10A90000401CC0B2A8710A2800D1AC71E879401C83
:10A91000C0B2E871322806D1EC71FCF753FCFEF7A7
:10A9200095FBFFF7D5F8287A401CC0B2287264283E
:10A9300006D12C72FAF7CEFBF9F7A4FAFCF7AEFCBD
:10A940006889401C80B26881B0F5967F0AD16C811D
:10A95000FEF752FCFEF7E2FCFEF71CFFFAF79CFC48
:10A96000FAF7B4F8A889401C80B2A881B0F5FA7F44
:10A9700006D1AC81FDF72EFFFAF7A8FDF8F71AFF14
:10A98000E889401C80B2E881B0F57A7F06D1EC817D
:10A9900000F00EF8FEF7CAFBF9F73CFBFBF7E2FF0D
:10A9A000FCF7E0FABDE87040FAF7F0BA5E03002069
:10A9B00070B51A4C0021A08800F05CFA2188814211
:10A9C00001D2491C03E019B1814201D9491E2180FD
:10A9D000E088134DB0F5E16F03D9012100F04AFA88
:10A9E000E8806088E988884201D2401C03E018B101
:10A9F000884201D9401E608020880A4A00EB80000E
:10AA00004FF6FF7101EA400022F84C0F608800EB1E
:10AA1000800001EA4000508070BD00001A00002054
:10AA2000C40000208C0200202DE9F0412A48407823
:10AA300040074FD529482B4D294C028928882A4B9D
:10AA400042B12178012905D19988C831884201D9BC
:10AA5000998000E098809E88B6F5596F00D2002654
:10AA6000217821480129C06809D142B140F6354119
:10AA700071431E4CB0EB411F01D302D808B94FF00F
:10AA80000504A0FB04011A4F98463A464FF0000314
:10AA9000F8F7BAFB391B714341181648B1FBF0F0C7
:10AAA00080B26880B0F52F7F01D800200FE0B0F5AC
:10AAB000616F02D341F2883009E041F28832A0F59B
:10AAC0002F70504340F6543290FBF2F080B2E88091
:10AAD000C8F80C10BDE8F08170030020900300203E
:10AAE00065020020F603002068000020AC8401000D
:10AAF000A0860100EB9207007047000010B5064CDD
:10AB000040F22551204600F009F82046BDE81040EB
:10AB100040F2277100F002B80044004070B501F027
:10AB20001F0501260024C1F3421306FA05F2012B8A
:10AB30000FD0022B0FD0838A4FEA112100881342D5
:10AB400006FA01F600EA060001D000B10124204611
:10AB500070BD8389F0E7038AEEE7000010B5114A63
:10AB600000211148F9F78AF80E48017A042914D116
:10AB70000C4C40681E3C010A60702170C0F30D400F
:10AB8000608004F1290000F0CFF82078002105282A
:10AB900004D0032801D10548418110BD04488183B8
:10ABA00010BD0000840500200064004090040020D7
:10ABB00070030020002904BF0020704730B4002338
:10ABC0004FF0010C0D461A4605E000BF4900521C2B
:10ABD0004FEA4C0CD2B2814298BF212AF6D34A08E0
:10ABE00000244FEA5C0C95420CD8904224BF801A96
:10ABF00063445208611C4FEA5C0CCCB2954298BF8A
:10AC0000212CF2D330BC18467047FEE7F0B51F4840
:10AC100000211F4A41704FF6FF70908050801D4800
:10AC20001F4A5F2341751C48214C81731B48E60372
:10AC300081721C48917303806E23438042F20F702F
:10AC4000508119484FF48072202301741748028004
:10AC5000012242808380C28004819503458153078D
:10AC6000C660C0E9043113489702078042808027FC
:10AC70008780C28004814581C660C0E904310E48E6
:10AC8000FF2120F8AC2FC182F0BD0000900400200D
:10AC90001C0400204C040020C4030020F603002004
:10ACA000900300201A00002070030020E004002020
:10ACB00000C0FFFFF80400208C020020154810B5EA
:10ACC000032100F8021F0022427001238370072431
:10ACD000C4700171427182710FA1C2710C6804626B
:10ACE0004C684462098901850E494FF6FF74498B0F
:10ACF00001EB810104EA4101C185022180F8A31022
:10AD0000A0F8B0304FF42F71A0F8BC10A0F8C2200A
:10AD100010BD00008C0200205A4552585F43414E3E
:10AD20005F3100001C0400201CB501788C0901F083
:10AD30003F018DF800408DF804104278837802EBD3
:10AD40000322084B92B21B7806D0012C07D0022CAC
:10AD500001D100F07DF91CBD00F020FA1CBD00F00F
:10AD6000E1F91CBD66050020F8B51E4EF07A0028FA
:10AD700020D0B1883289881A83B230460024006816
:10AD80001AB1072B17D9072516E0164A0529C9B2AB
:10AD9000D2884FF00003009203D8002200F008FC94
:10ADA0001DE0012200F004FCB088052800D9052030
:10ADB0003081B472F8BDDDB210440094B37A02223F
:10ADC000294600F0F5FB3089284480B23081B17A01
:10ADD000491C01F00F01B172B1888842EAD3F472C4
:10ADE000F8BD000010050020094A002101EB4103D5
:10ADF00032F81330834204D101EB410002EB4000F2
:10AE00007047491C89B22C29F0D3002070470000FC
:10AE10009AC2000814488078C2071448C1880CD030
:10AE200040F2DC52808A914217D9104A40F6AC5366
:10AE30009942928C07D310460FE00D4A527800EBEE
:10AE40004200408A09E0121AA1F2DC535A434FF43F
:10AE5000FA6392FBF3F2104480B241434FF47A70EC
:10AE600091FBF0F000B2704770030020F603002061
:10AE700090040020002247F6F813984284BF002077
:10AE8000704730B401230E4C04F5217500290CBF26
:10AE900054F822C055F822C0844504D3521C5B1CD0
:10AEA00092B2A22BF2DD00291EBF104630BC7047C3
:10AEB000282A86BFA2F1280080B2002030BC70474B
:10AEC000F4C600082DE9F04F574B0027574DB3F853
:10AED00008C04FF4FA61BCF1000F1DD06F81B5F9C5
:10AEE0000600DFF84CA1C0EB8012544CBAF9000008
:10AEF000DFF84091104480112881B5F80A808B4614
:10AF00004D4EB4F91010A289B9F81400D8450BD2EF
:10AF1000BCF1000F06D008E068898842DFD2401CEF
:10AF20006881DCE73C2800D382B194F80AC0BCF108
:10AF3000000F0BD093F8323003B13AB1404AD278C7
:10AF4000D20603D43F4AB2F8C42072B1B6F9000069
:10AF5000814200DD2082B4F91000B0F5807F02DD6F
:10AF6000A0F5807055E0278254E04FF4C8729142FA
:10AF700000DA2282FFF74EFF334980B220810F7042
:10AF8000B5F90810884225DDA0EB0100B9F80A20C8
:10AF90002E49C0F38F000A2A02D94978183103E0FC
:10AFA0004A78082101EB5201814200D20846B4F9E7
:10AFB0001020B6F900108A4200DA2182B4F910108C
:10AFC000594503DA4FF6FF7202EA800000B901200A
:10AFD000084415E017DA081AC0F38F00082801D9D1
:10AFE000082001E000B90120B4F91020B6F90010E2
:10AFF0008A4200DD2182B4F91010814202DD081A74
:10B00000208200E02782B4F91000E189884201DD46
:10B0100088B22082A08908B1401EA081BAF8000041
:10B02000E880BDE8F08F0000900300206800002059
:10B03000EA0000201C04002068020020F603002023
:10B04000700300208C0200202200002090040020C9
:10B0500070B5314D95F84720002A5BD095F8462011
:10B060008A4251D1B5F84010B5F84230C91A8AB2B7
:10B07000072A01D9072400E0D4B22B44411C224600
:10B080001846F8F738F9B5F84200204480B2A5F820
:10B09000420095F84610491C01F00F0185F8461052
:10B0A000B5F84010884235D3B5F84400FFF79CFE50
:10B0B000040029D0E07838BBA0881849B5F84020B2
:10B0C000461815493046F8F716F9B5F84000A1784A
:10B0D000884204D2091A30442022F8F751F9B5F811
:10B0E0004400042806D0A0F58071573902D0B0F58D
:10B0F000AC7F02D10A4A0121D17095F8483095F809
:10B100004020054900F0B4FABDE870404A210248E9
:10B11000F8F73EB970BD00001C0500208C0200202D
:10B12000280000202DE9F047814698460F46164634
:10B130001046FFF759FE05002CD0174C94F8470035
:10B1400018B14A212046F8F723F9A978B81E891CBE
:10B150003E281FD28F421DD880B2A4F84000052897
:10B1600001D9052100E0014624F8421F0021668034
:10B1700021710121617184F8068000280AD0052818
:10B1800000D9052009F10301BDE8F047C2B2024829
:10B19000F8F7B1B8BDE8F0871C0500202DE9F05F95
:10B1A00007469B460D4616461046FFF71DFE040057
:10B1B0003DD02C4890F8470018B14A212948F8F7AB
:10B1C000E7F829494FF000094FF0010A022D1CD081
:10B1D000E07800282BD1AD1EA078EDB2A84200D2B5
:10B1E0000546A0882A4608448046F91CF8F783F8EB
:10B1F000A078A84205D9411B08EB05002022F8F7EA
:10B20000BFF8B6F5887F14D024E0A0880144154823
:10B210000C380160A1788180C680A0F8089013499D
:10B2200080F80A9080F80BA081F801B08E80BDE80C
:10B23000F09F0F4A907868B90E48A0F81890C0F8AF
:10B240000890046943682344C0E90093C0F8109053
:10B2500082F802A05B462A46F91C3046BDE8F05F42
:10B2600000F006BA1C0500208C0200203C000020E3
:10B27000280000209C04002072B64FF440514FF08B
:10B280000060FEF743FBFCF701F8FFF7BFFCFFF798
:10B2900015FDF9F741FBF8F7EDFAFDF77FFAF9F73D
:10B2A00060FE62B6F9F76AFEFFF7FCFAFCE7000001
:10B2B0002DE9F04F6A4F0122B7F802A0BAF5BA5F44
:10B2C00038BFBA73674801896748B0F8068031B95A
:10B2D0006448B8F1640F8273634838BF82724FF0DC
:10B2E000000C6249624D81F800C081F801C081F80C
:10B2F00002C028785F4B604C0128B3F916B09E8AD3
:10B3000007D00A2E05D8BBF10A0FDCBFE27784F81C
:10B310001EC05A4890F8009049F0400980F800900B
:10B3200095F800E05648BEF1000F04BFB4F80EE0F7
:10B33000BEF1000F7ED1B4F906E0BEF10A0FA4BF42
:10B3400094F80DE0BEF1000F7CD1B3F818E0AEF137
:10B35000050EF34576DA94F803B01BF0100F71D1A7
:10B36000DFF820E1BEF8C4E0BEF1000F6AD19B8B8C
:10B3700006F11E0E9E4565D21BF0010F4FF0020B29
:10B3800001D1237C13B185F800B05BE0354B5C7BC9
:10B39000002C08BF5A73394C6478002C52D0364CBC
:10B3A000647814F0010F1EBFBF7B002FBAF5BA5F9F
:10B3B0000DD919F0400F01D01E2E08D90A70067859
:10B3C000761CF6B20670032E28BF85F800B02A4F0F
:10B3D000244E14F0020F367B1CBF93F80E90B9F187
:10B3E000000F11D093F80D90B1450DD84A7090F828
:10B3F000019009F1010909F0FF0980F80190B9F104
:10B40000030F28BF85F800B014F0040F18D0164CB5
:10B41000A47AACB15B7B9E4212D3BB7F002B14BFDE
:10B4200064234FF4966343450AD28A708278521C93
:10B43000D2B200E006E08270032A28BF85F800B08F
:10B440000A780AB980F800C04A78002A08BF80F854
:10B4500001C08978002908BF80F802C0BDE8F08FDC
:10B46000C403002090030020F603002057000020B2
:10B47000650200201C0400207003002090040020BE
:10B48000540000208C02002030B5174D174C28784E
:10B4900058B12089A080E080A08840F6AC510022FD
:10B4A000884205D3A28222820EE0F8F7BDF9F3E7C5
:10B4B000218801EBC1018900B1FBF0F1A1824EF6B8
:10B4C0006021B1FBF0F02082B4F91000002809DD02
:10B4D000B4F90E1000EB8000C901400091FBF0F0C0
:10B4E000A88030BDAA8030BD4C0400201C04002080
:10B4F0002DE9F04706462C4885696988B14201D399
:10B5000028880CE0007F6FF0010101EB8002AA5A4D
:10B510006FF00308B24206D808EB8000285ABDE855
:10B52000F04700F0EDBC0124022738E007EB84026D
:10B53000AA5AB24231D901EB8400285A00F0E0FC4B
:10B54000814608EB8400285A00F0DAFC804607EBBD
:10B550008400285A00F0D4FC074635F8240000F097
:10B56000CFFC04464946384600F0AAFD0546414650
:10B57000204600F0A5FD0446304600F0C1FC4946D7
:10B5800000F09EFD214600F0CFFC294600F0D6FBDE
:10B590004146BDE8F04700F06FBB641CE4B2A04236
:10B5A000C4D80248BDE8F087640400200000C84207
:10B5B0002DE9F041DFF8ACC00424069D8CF808406A
:10B5C000294E00248CF80940778896F800E03F0463
:10B5D000767807EB0E273E44CCF8046008268CF8FA
:10B5E0000A60ACF16006EFB246F86B4F74608C1CD9
:10B5F0002E0A04F03F040CF10E0522B1012A0CD0F2
:10B60000022A28D116E08CF80B400AE018B305296D
:10B610000ED80A46014628461BE044F040028CF84A
:10B620000B208CF80C708CF80D600029EED112E024
:10B630000521EEE703F00F0242F080028CF80B20A8
:10B6400049B140B1072900D907210A4601460548FA
:10B650000C30F7F750FEBDE8F04102490348F8F717
:10B660004CBB0000700500203C000020006400403E
:10B6700070B51D4614460646402A00D9402422468D
:10B680000848F7F738FE0748A0F1880108608C8069
:10B69000CE800020088188720120C872024845705F
:10B6A00070BD0000980500203C00002002494FF0CA
:10B6B000000000F07ABD00BF0000F87F2DE9C04116
:10B6C00030B4DFF8A0C23CEA111418BF3CEA1314EE
:10B6D00000F0EC8081EA03051CEA111444EAD574F9
:10B6E00018BF1CEA131500F0C780A4EB05044FF047
:10B6F000004545EAC12145EAC32341EA505143EAE6
:10B70000525304F17F74994204F500344FEAC0208B
:10B710004FEAC22208BF904200F09C804FEA1365B6
:10B720000FF24016765D4FEA134506FB05F7C7F1A9
:10B73000807706FB07F74FEAD737A7FB0368764207
:10B74000C8F58038A7FB06CE38BFA8F1010807FB73
:10B7500008E64FF0000EA6FB028CE6FB03CEDCF100
:10B76000000CCEF1004E38BFAEF1010EA6FB0C5816
:10B770004FF000074FF00005E6FB0E87A1FB08C65F
:10B78000A0FB07CE16EB0E0645F10005E1FB0765B1
:10B7900015F1E04E7EBFA4F580345FEA46066D41A8
:10B7A00016F1800745F100054FEA17274FEA0666B4
:10B7B00047EA0567A6F1DE46B6F1805F4FEA152538
:10B7C0001FD9384624F0010C05EBC471BCF1FE6FA3
:10B7D00001EB0C1102D8F0BCBDE8008124425CBF33
:10B7E00001F5801E9EEAC47F02D4F0BCBDE8008152
:10B7F000244238D4F0BCA1F1C041BDE8004100F0C2
:10B8000035BA4FEAD22242EA43524FEAD323A7FB8A
:10B8100002864FEAD02040EA415007FB03661EEA49
:10B820000E0F4FEAD12105FB026658BFA6EB00566A
:10B83000B6EB00564FEA520E4EEAC37E18EB0E0EE0
:10B8400056EB530EBDD518EB02085E417F1C55F137
:10B850000005B6E74FF480154FF000074FF00006E3
:10B860004FF00008ADE7F0BC4FF0000001F1C0411F
:10B8700001F00041BDE8008111EA0C1F0CEA13152C
:10B8800000D00CE013EA0C1F00F025804FF0000000
:10B89000F0BC81EA030101F00041BDE80081F0BC89
:10B8A000BDE8004181EA030100F0E0B9F0BCBDE869
:10B8B000004170B500F08CF9097EFC3E00F007B83D
:10B8C00081EA03014FF0000001F00041704781EA76
:10B8D000030100F0CBB9F0BCBDE800414FF000001F
:10B8E00021497047FFFDFBF9F7F5F4F2F0EEEDEBBF
:10B8F000E9E8E6E4E3E1E0DEDDDBDAD8D7D5D4D36E
:10B90000D1D0CFCDCCCBCAC8C7C6C5C4C2C1C0BFB9
:10B91000BEBDBCBBBAB9B8B7B6B5B4B3B2B1B0AFBF
:10B92000AEADACABAAA9A8A8A7A6A5A4A3A3A2A1A3
:10B93000A09F9F9E9D9C9C9B9A999998979796955E
:10B9400095949393929191908F8F8E8E8D8C8C8BFA
:10B950008B8A898988888787868585848483838282
:10B96000828181800000FF070000F87F4FEA4103D9
:10B970004FEA5353A3F58063D3F11E03C8BFD3F13D
:10B98000210C0CDD4FF0004242EAC12242EA505243
:10B9900032FA03FC8CEAE17CACEBE1707047102BCF
:10B9A000C4BF0020704703F5787CBCF1FF3F04D092
:10B9B0006FF0004282EA2100704770B500F008F98C
:10B9C0004992248000207047F2E700004FEA1153AB
:10B9D000A3F58063D3F11E03A8BFD3F1200C08DBCD
:10B9E0004FF0004242EAC12252EA505232FA03F0CA
:10B9F000704709420BD4102BC4BF0020704703F5D9
:10BA0000787CBCF1FF3F05D04FF0FF3070474FF01E
:10BA10000000704770B500F0DBF800BF4992248049
:10BA200000207047F0E710F0004248BF4042B0FAF3
:10BA300080F310FA03F10AD0C3F11D0303F580630C
:10BA40004FEA415002EB035202EBD12170474FF015
:10BA500000007047B0FA80F310FA03F10AD0C3F186
:10BA60001D0303F580634FEA41504FEA035202EB96
:10BA7000D12170474FF0000070470000DFF848C147
:10BA800070B51CEA111E1EBF1CEA13159EEA0C0FAE
:10BA900095EA0C0F00F06F8081EA030423EA4C134F
:10BAA0004EEAD47E21EA4C1141F4801143F4801314
:10BAB000AE44A1FB024CA0FB0365AEF17F7E3619BC
:10BAC00055EB0C05A1FB034C4CF10003A0FB021C41
:10BAD00016EB0C06654153F10003094218BF46F00E
:10BAE000010613F4007F0BD14FEA03314FEA053012
:10BAF000340341EA155140EA16506FF003020AE0A0
:10BB00004FEAC3214FEAC520F40241EA555140EA09
:10BB100056506FF0020202EB2E4201EB025585EA0D
:10BB2000CE710AD05FEA440C18BF24F0004450F1F3
:10BB3000000041F1000120EAD47040F2FE7C624531
:10BB400000D270BDA84214BF4FF080444FF0404473
:10BB5000002E08BF0024BEF1806FA8BFA1F1C04134
:10BB6000BDE8704080F282804FF0000001F1C041DA
:10BB700001F0004170479EEA0C0F0CEA131518BF44
:10BB800095EA0C0F06D04FF0000081EA030E0EF08C
:10BB9000004170BD00F01CF88900013E00F007B8BC
:10BBA00000F009B84FEA430C5FEA5C5C08D081EA18
:10BBB000030100F05BB84FEA410C5FEA5C5CF6D130
:10BBC0004FF00000014970470000FF070000F87FB8
:10BBD0000EF1020E2EF0030E5EF8046B364205D411
:10BBE000012A43EB030515F5001F12D8012841EB8C
:10BBF000010C1CF5001F0CD80ED14FEAD17C15F5B5
:10BC0000001F0CEB4C0C0CF1020C08BF4CEBD37C6E
:10BC100004E04FF0080C01E04FEAD37C0CEB4C053C
:10BC200026FA05F606F00706B6F1040C06D20EEB6E
:10BC3000860CBDE870404CF0010C6047DFE80CF06A
:10BC4000090B02024FF000414FF00000A1F5002166
:10BC500070BD19461046012851EB010418BFD4F5F8
:10BC6000001484BF002001F0004170BD0808A0F559
:10BC700000114FEA3101704790EA010F48BF81F08F
:10BC8000004100F12482421A3CBF801A89184FEA11
:10BC9000D0524FF07F4C1CEA410FA2EBD15318BF9A
:10BCA0009CEA026F00F03B804FF0004C4CEA002011
:10BCB0004CEA012121FA03FC10EB0C0C1ED202F11C
:10BCC000FF325FEA1C2040EBC25038BF70471CF0C7
:10BCD0007F0F4FEA400C18BFBCF17F4F38BF704751
:10BCE000C3F12003994008BF20F00100BCF17F4F51
:10BCF00038BF7047A0F1C04000F0DDB94FEA3C000A
:10BD0000000A40EBC25028BF1CF0FF0F4FEA400C66
:10BD1000E6D018BFBCF17F4F38BF7047EAE79CEA16
:10BD2000026F05D010EA5C0F08BF00F000407047BA
:10BD300010B500F07AF900BF64FBBE3E4FF47F0CF3
:10BD40001CEAD0121EBF1CEAD11392EA0C0F93EA30
:10BD50000C0F00F0858090EA010F48BF42F480721A
:10BD600040F4000C41F400002CF07F4120F07F40B3
:10BD700000B58142A2EB03020FF2081CACEB504E5F
:10BD8000C0F100009EF800E04FEA4E0E00FB0EFCF2
:10BD900038BF49004FEA2C1C02F5FA020CFB0EF3E7
:10BDA0004FEACE1E4FEA112C4FEAC1210EEB635E23
:10BDB00042EB22420EFB0CFC4FEA1C5300FB03112A
:10BDC0004FEA112C4FEA01310EFB0CFC4FEADC4C20
:10BDD00000FB0C11C14228BF09184CEB03335DF87E
:10BDE00004EB10EB410143EBC250B2F57C0F38BFBE
:10BDF000704729D512F0F00F1CBF00F1C04000F0D1
:10BE000000407047008182838485868788898B8C77
:10BE10008D8E8F919293959697999A9C9D9FA0A2B3
:10BE2000A3A5A7A8AAACAEB0B2B3B5B7B9BCBEC003
:10BE3000C2C5C7C9CCCED1D4D7D9DCDFE2E6E9ECA4
:10BE4000F0F3F7FAFE0000004FEA400C0CF1807CA2
:10BE5000BCF17E4F28BF7047B0F1C04000F02BB955
:10BE600090EA010F0CEAD11348BF42F48072624598
:10BE700038BF634507D213F47F0F16D080EA010064
:10BE800000F00040704710B500F0CFF8097EFC3E8E
:10BE900000F005B880EA010000F00040704780EA39
:10BEA000010000F0004000F006B912F47F0F04BF5B
:10BEB0000248704780EA010000F0FDB80000C07F32
:10BEC000C10DD1F19E0206DB4FEA002343F000438F
:10BED00023FA02F07047004207D54FEA4001B1F162
:10BEE000FE4F02D24FF00000704710B500F09DF8F1
:10BEF00049922480002070476FEA200070470000BC
:10BF0000B0FA80F310FA03F2C3F19D030AD0D90509
:10BF100001EB1220530638BF704700F1010008BF43
:10BF200020F00100704700004FF47F0C1CEAD01293
:10BF30001EBF1CEAD11392EA0C0F93EA0C0F00F01B
:10BF4000478090EA010F48BF42F480724FF0004CE6
:10BF50004CEA00204CEA012102EB0302A0FB011392
:10BF6000A2F50002002918BF43F001035B0028BFBF
:10BF70004FEA330342EB22425FEA132C4CEBC250F0
:10BF80002EBFBCEB436FB2F57C0F70474FEA036CDA
:10BF9000BCF1004F08BF20F00100B2F57C0F38BFA4
:10BFA00070470BD582F0FF0212F5803FC8BF704783
:10BFB00000F1C040D8BF00F00040704700F5000C11
:10BFC0005FEA4C0C48BF7047B0F1C04000F073B856
:10BFD00090EA010F0CEAD11348BF42F48072624527
:10BFE00038BF634504D280EA010000F0004070478A
:10BFF00010B500F01AF800BF8900013E00F007B844
:10C0000000F009B85FEA410C5FEA1C6C08D080EAD6
:10C01000010000F050B85FEA400C5FEA1C6CF6D1FA
:10C020004FF00040A0F5800070470EF1020E2EF098
:10C03000030E5EF8044B244204D44FEA4102B2F1ED
:10C040007F4F11D84FEA4003B3F17F4F0CD80ED188
:10C050004FEAD07CB2F17F4F0CEB4C0C0CF1020C90
:10C0600008BF4CEBD17C04E04FF0080C01E04FEA34
:10C07000D17C0CEB4C0324FA03F404F00704B4F174
:10C08000040C06D20EEB840CBDE810404CF0010C01
:10C090006047DFE80CF0070802024FF00040A0F50F
:10C0A000800010BD0846420018BFD2F1807288BFE0
:10C0B00000F0004010BDFF2141EAD050C00570479C
:10C0C00090EA010F48BF81F000413FF5DCAD421A14
:10C0D00004D882F00042A0EB020011444FEAD05293
:10C0E0004FF07F4C1CEA410FA2EBD15318BF9CEAE2
:10C0F000026F4AD04FF0004C4CEA00204CEA01217C
:10C1000021FA03FCB0EB0C0C0FD412F0FE0F36D06A
:10C110005FEA4C001DD5001240EBC25038BF70479B
:10C120001CF03F0F18BF70470BE0A2F101025FEA5D
:10C130001C2040EBC25038BF70471CF07F0F18BF67
:10C140007047C3F12003994014BF401E20F0010046
:10C15000704780084FEA122308BF7047B0FA80FC8E
:10C16000A2EB0C02CCF1280C60FA0CF093EA122F2F
:10C1700004BF00EBC25070474FEAC3707047130A08
:10C180005FEADC1008BF7047F6E79CEA026F04D054
:10C1900010EA5C0F08BF0020704710B5FFF745FF9D
:10C1A00040DFF63E81F0004070470CF00F03092B92
:10C1B00008BF082000F059800A2B0BD0082B18BFAD
:10C1C000704708BF1CF0400F0AD04FF000004FF03E
:10C1D000000170471CF0400F18BF4FF0004070473F
:10C1E0001CF0100F08D020F0704300F07F4242EAAC
:10C1F000D3014FEA4370704700F0604021F07F4266
:10C2000042EA000201F07F4040EA727070474FF04E
:10C21000FF0C4CF4E06C1CEA11531CBF9CEA030CAD
:10C220009445C2BFDA4201EB02517047002B0DD09A
:10C23000BCF1000F0FD0002A01F00041A4BF41F073
:10C24000E04141F07F614FF00000704701F0004194
:10C250004FF00000704750EA01334FF09B0C18BFBD
:10C260004CF0806C7FF422AA70471CF4801F11D020
:10C270001CF4E02F03D06FEACC31490070474FF037
:10C280004050EFF3008222F0704242EA000282F353
:10C29000008870474FF00000704701000201000065
:10C2A000020004010200030004010600040018005B
:10C2B0000A0005000A012200070002002C0000010C
:10C2C00002002E00020102003000030102003200D1
:10C2D0000D010401340010010400380011010401B3
:10C2E0003C001F01040140006001040144001007EC
:10C2F00002014800110702014A00001102014C002E
:10C30000021102014E0006F10A01970005F1040036
:10C31000A10007F10400A50024010200A90004FF08
:10C320000100AB0059010201AC00001902005200EB
:10C3300025020400AE0020020200B4000601020043
:10C34000B20021020200B60023020400B800570127
:10C3500015005300580115006800140118007D00F5
:10C360000B09020195001318020150001209020185
:10C37000BC0011090201BE0019010200C6001D180F
:10C380000401C8001E180401CC001A010200C400F8
:10C3900013010201C00007F50200C20020190201CA
:10C3A000D0000000E8080500060908004C090A0052
:10C3B0007409140092091E00C4092800D80932002B
:10C3C000000A3C00460A4B008C0A5A00D20A64005C
:10C3D000220B0000B20C0500E40C0800480D0A0016
:10C3E0007A0D1400AC0D1E00E80D2800100E32006E
:10C3F000420E3C00A60E4B000A0F5A006E0F64005E
:10C40000041000003C0F0500780F0800F00F0A0030
:10C410002C10140068101E00B8102800E010320024
:10C420001C113C0094114B000C125A008412640041
:10C43000F21200003610050068100800FE100A0015
:10C44000C6111400F8111E00481228008E12320086
:10C45000CA123C0056134B00CE135A001E1464003F
:10C460008214000094110500D011080048120A003F
:10C470008E121400D4121E0024132800561332000A
:10C480009C133C001E144B00A0145A0018156400A5
:10C490007C15000050140500A01408002C150A009B
:10C4A0007C151400CC151E003016280076163200BC
:10C4B000C6163C005C174B00E8175A006A18640067
:10C4C000CE1800006A180500CE18080078190A0076
:10C4D000DC191400401A1E00B81A2800081B32008C
:10C4E0006C1B3C00201C4B00D41C5A007E1D6400B9
:10C4F000141E00000000C90092015B022403ED033A
:10C50000B6047F0548061107D907A2086B09330A4C
:10C51000FB0AC40B8C0C540D1C0EE40EAB0F7310F5
:10C520003A110112C8128F1355141C15E215A816E2
:10C530006E173318F918BE19831A471B0C1CD01C30
:10C54000931D571E1A1FDD1F9F2062212422E52202
:10C55000A72367242825E825A82668272728E52873
:10C56000A429622A1F2BDC2B992C552D112ECC2EA1
:10C57000872F4230FC30B5316E322733DF339734AA
:10C580004E350436BA3670372538D9388D39403AA9
:10C59000F33AA53B573C083DB83D683E173FC63FC0
:10C5A00074402141CE417A422643D1437B44244505
:10C5B000CD4575461D47C4476A480F49B449584A96
:10C5C000FB4A9E4B404CE14C814D214EC04E5E4F8C
:10C5D000FB4F98503451CF51695203539B533354FE
:10C5E000CA546055F6558A561E57B1574358D45809
:10C5F0006459F459825A105B9D5B295CB45C3E5DC2
:10C60000C85D505ED75E5E5FE45F6860EC606F613E
:10C61000F1617262F2627163EF636C64E964646594
:10C62000DE655766D0664767BD673268A7681A69D6
:10C630008C69FD696E6ADD6A4B6BB86B246C8F6C1C
:10C64000F96C626DCA6D316E976EFB6E5F6FC26F73
:10C6500023708370E37041719E71FA715572AF72ED
:10C6600008735F73B6730B746074B3740575567595
:10C67000A675F47542768E76D97623776C77B47783
:10C68000FB7740788578C8780A794A798A79C979B8
:10C69000067A427A7D7AB77AEF7A277B5D7B927B46
:10C6A000C67BF97B2A7C5A7C897CB77CE47C0F7D35
:10C6B0003A7D637D8A7DB17DD67DFB7D1E7E3F7E8A
:10C6C000607E7F7E9D7EBA7ED67EF07E0A7F227F50
:10C6D000387F4E7F627F757F877F987FA77FB57F8A
:10C6E000C27FCE7FD97FE27FEA7FF17FF67FFA7F3C
:10C6F000FE7FFF7FF8790000A279000048790000F2
:10C70000EA7800008878000022780000B8770000FE
:10C7100049770000D67600005E760000E1750000E3
:10C7200060750000DA7400004F740000BE730000F2
:10C73000297300008F720000EF7100004A71000041
:10C74000A0700000F06F00003B6F0000806E0000E2
:10C75000C06D0000FA6C00002F6C00005F6B0000E1
:10C76000896A0000AD690000CD680000E76700003D
:10C77000FB6600000B660000156500001B640000EE
:10C780001C630000186200000F61000002600000DE
:10C79000F15E0000DC5D0000C35C0000A65B0000F1
:10C7A000855A0000615900003A58000010570000F7
:10C7B000E3550000B4540000825300004F520000C3
:10C7C0001A510000E34F0000AB4E0000724D000014
:10C7D000384C0000FE4A0000C349000088480000B1
:10C7E0004E47000014460000DA440000A243000057
:10C7F0006A4200003441000000400000CD3E0000CD
:10C800009C3D00006D3C0000413B0000173A0000D9
:10C81000F0380000CB370000AA3600008B3500004E
:10C8200070340000583300004432000033310000FF
:10C83000263000001D2F0000172E0000162D0000CE
:10C84000182C00001F2B0000292A000038290000A6
:10C850004A280000612700007C2600009B2500007C
:10C86000BF240000E6230000122300004122000044
:10C8700075210000AD200000EA1F00002A1F000003
:10C880006E1E0000B71D0000031D0000531C0000B9
:10C89000A71B0000FF1A00005A1A0000BA19000076
:10C8A0001D19000083180000EE1700005B17000040
:10C8B000CC16000041160000B91500003415000028
:10C8C000B214000033140000B81300003F1300003E
:10C8D000C912000057120000E71100007A11000091
:10C8E0000F110000A710000042100000E00F000030
:10C8F000800F0000220F0000C60E00006D0E000029
:10C90000160E0000C20D00006F0D00001F0D00008C
:10C91000D00C0000840C0000390C0000F10B00006A
:10C92000AA0B0000650B0000220B0000E00A0000CB
:10C93000A00A0000620A0000250A0000EA090000BF
:10C94000B109000079090000420900000D0900004A
:10C95000D8080000A6080000740800004408000081
:10C9600015080000E7070000BB0700008F07000064
:10C97000650700003B0700000A7C0000E07B000028
:10C98000AE7B00007A7B0000437B00000A7B000046
:10C99000CF7A0000927A0000527A00000F7A0000ED
:10C9A000BC7900008279000038790000EB78000043
:10C9B0009A78000047780000F1770000987700002F
:10C9C0003B770000DC7600007976000012760000EC
:10C9D000A87500003B750000CA7400005674000082
:10C9E000DE73000062730000E27200005F720000FC
:10C9F000D87100004D710000BE7000002B70000067
:10CA0000946F0000FA6E00005B6E0000B86D0000CD
:10CA1000126D0000676C0000B86B0000056B000031
:10CA20004F6A000094690000D66800001368000097
:10CA30004D67000082660000B4650000E3640000FA
:10CA40000D6400003463000058620000786100004B
:10CA500094600000AD5F0000C35E0000D65D000082
:10CA6000E65C0000F25B0000FC5A0000045A000083
:10CA7000085900000A5800000A5700000856000034
:10CA800003550000FC530000F4520000E95100007F
:10CA9000DE500000D14F0000C24E0000B34D000038
:10CAA000A34C0000914B00007F4A00006D4900003C
:10CAB0005A48000047470000354600002145000065
:10CAC0000F440000FD420000EC410000194000004E
:10CAD000CB3F0000BB3E0000AD3D0000A13C00008C
:10CAE000953B00008C3A0000843900007E3800003D
:10CAF0007A37000077360000773500007A3400007E
:10CB00007E33000085320000D83000009A300000EB
:10CB1000A92F0000BB2E0000D02D0000E62C000045
:10CB2000012C00001F2B00003F2A0000612900009B
:10CB300089280000B2270000DF260000112600002F
:10CB4000452500007A240000B5230000F3220000F0
:10CB50003422000079210000BF2000000A200000DC
:10CB60005A1F0000AB1E0000001E0000591D0000EF
:10CB7000B51C0000121C0000761B0000DB1A000030
:10CB8000431A0000AD1900001C1900008F180000A6
:10CB9000031800007B170000F51600007216000055
:10CBA000F215000076150000FD1400008614000048
:10CBB000121400009F13000030130000C312000085
:10CBC0005A120000F21100008C1100002A1100001E
:10CBD000CA100000691000000F100000B50F00001F
:10CBE0005C0F0000060F0000B40E0000610E000094
:10CBF000110E0000C30D0000770D000008080808A2
:10CC0000080808080808000028CC000800000020D8
:10CC10008C02000028310008A8CC00088C020020FB
:10CC20008C160000843100081184D8B8050009284A
:10CC30000102030406070809120103269C1C022DA9
:10CC400046EBFFFF10091C016102496E32065A07CC
:10CC5000045A0510E908291CE92829046910091259
:10CC6000346920E9280110032001010318CF03884B
:10CC7000099E07DA16B42DDA160201160C17B0CA8F
:10CC80000B66180807030602050104A91009030131
:10CC90000604020706041B05020B140601050C120C
:08CCA000030204B3014500008A
:04000005080030EDD2
:00000001FF
